:020000040000FA
:040200006BEF03F0AD
:040208000EEF01F004
:080218002DEF01F0D8CF01F039
:10022000E0CF02F0006EF3CF03F0F4CF04F0F0ACB7
:100230001DEF01F0F0B066EC0BF0A2A023EF01F08F
:10024000A1B018EC09F003C0F3FF04C0F4FF0050A4
:1002500002C0E0FF01C0D8FF1000D8CF06F0E8CF01
:1002600005F0E0CF07F0F3CF08F0F4CF09F0F0BCD1
:100270003DEF01F0F0B066EC0BF0A2B043EF01F0FF
:10028000A1B018EC09F0A2B04CEF01F0AECFE8FF3E
:100290006ECFE8FF52EF01F09EBAFCEC0EF0A4BA6C
:1002A00067EC0FF008C0F3FF09C0F4FF07C0E0FFE0
:0A02B00005C0E8FF06C0D8FF1000EB
:10030000F95000011150F926BEEF29F0C0EF29F095
:10031000CDEF29F0E2EF29F0F0EF29F0FEEF29F020
:100320000CEF2AF01AEF2AF02AEF2AF038EF2AF021
:1003300046EF2AF012000009D8A4A5EF01F0000151
:10034000000E0F6E000E106E1200E806030B0A0D71
:10035000F9CFE8FFF350F92683C00FF084C010F006
:10036000120085C00FF086C010F0120087C00FF099
:1003700088C010F0120089C00FF08AC010F012007F
:10040000EFCFE8FFE806070B0A0DF9CFE8FFF3503E
:10041000F9263CC04EF03DC04FF012003AC04EF0FD
:100420003BC04FF012003EC04EF03FC04FF01200F4
:1004300040C04EF041C04FF0120042C04EF043C0E9
:100440004FF0120044C04EF045C04FF0120046C0BD
:100450004EF047C04FF0120048C04EF049C04FF078
:1004600012000F0B060DF9CFE8FFF350F926BBC2BF
:10047000E8FF1200BCC2E8FF1200BDC2E8FF120094
:10048000BEC2E8FF1200BFC2E8FF1200C0C2E8FF10
:100490001200C1C2E8FF1200C2C2E8FF1200C3C2CC
:1004A000E8FF1200C4C2E8FF1200C5C2E8FF120054
:1004B000C6C2E8FF1200C7C2E8FF1200C8C2E8FFC8
:0E04C0001200C9C2E8FF1200CAC2E8FF120013
:100500000001E806070B0A0DF9CFE8FFF350F926C2
:100510008D510D6E8E510E6E12008F510D6E9051D9
:100520000E6E120091510D6E92510E6E120093518B
:100530000D6E94510E6E120095510D6E96510E6E09
:10054000120097510D6E98510E6E120099510D6E5A
:100550009A510E6E12009B510D6E9C510E6E120040
:100600000001E8BE33EF03F0E806070B0A0DF9CF4F
:10061000E8FFF350F9260D5073270E507423120093
:100620000D5075270E50762312000D5077270E506F
:10063000782312000D5079270E507A2312000D50A6
:100640007B270E507C2312000D507D270E507E23F9
:1006500012000D507F270E50802312000D5081276D
:100660000E5082231200E806070B0A0DF9CFE8FFAF
:10067000F350F9260D50736F0E50746F12000D5029
:10068000756F0E50766F12000D50776F0E50786FA9
:1006900012000D50796F0E507A6F12000D507B6F63
:1006A0000E507C6F12000D507D6F0E507E6F120049
:1006B0000D507F6F0E50806F12000D50816F0E50E5
:1006C000826F1200F2AE12000001010EA16FA1674D
:1006D00067EF03F0120092988088939C819C000140
:1006E0005B6A5C6A640E9DEC0BF092988088000156
:1006F000546A640E9DEC0BF00F018350306E316E26
:10070000326E0F018450336E346E356E0F01999046
:10071000878094969394829681940001000E176EC0
:10072000000E186E0001000E196E000E1A6E000108
:10073000000E1B6E000E1C6E0001000E1D6E000EE2
:100740001E6E0001000E136E000E146E0001000EEE
:10075000156E000E166E0001000EAB6F000EAC6F32
:100760000001000EAD6F000EAE6F0001000EAF6F06
:10077000000EB06F0001000EB16F000EB26F0001ED
:100780005E6A5F6A606BA16BA26BA36BE769E96B42
:100790000201BA6B0101116B0001CC6B81EC31F0ED
:1007A000020100510001A56F040E93EC08F0040E45
:1007B00093EC08F00001C350C56FC450C66F050E1E
:1007C00093EC08F0050E93EC08F00001C350C76FDE
:1007D000C450C86F000EE8CF0DF0E86AE8CF0EF005
:1007E000A8EC0BF0E8CF00F5010EE8CF0DF0E86AB9
:1007F000E8CF0EF0A8EC0BF0E8CF01F5C0EC0CF060
:10080000FA0E9DEC0BF0FA0E9DEC0BF0FA0E9DEC3F
:100810000BF0FA0E9DEC0BF0C8EC08F0B7EC24F0EE
:1008200095EC0EF0A9EC0EF0F28EF28CD08E0F014A
:10083000D89083B6D880D8B023EF04F00A0E9DEC90
:100840000BF00F01D89083B6D880D8B039EF04F000
:100850000F01D89084B2D880D8B034EF04F00A0EDB
:100860009DEC0BF00F01D89084B2D880D8A05BEF3C
:1008700004F084EC1EF00201A50EA76346EF04F01D
:10088000E70EA86346EF04F04AEF04F081EC31F084
:10089000C9EC0BF000C2E8FFFFEC1EF00301AD5104
:1008A0000201A56FE9EC0AF064EC0AF00101F20E16
:1008B000066FA1EC0AF00F01D89084B2D880D8A0BE
:1008C0005BEF04F00A0E9DEC0BF00F01D89084B2A0
:1008D000D880D8A05BEF04F00F01D89084B4D88002
:1008E000D8B078EF04F00A0E9DEC0BF00F01D89011
:1008F00084B4D880D8B08EEF04F00F01D89083B6BE
:10090000D880D8B089EF04F00A0E9DEC0BF00F01EF
:10091000D89083B6D880D8A0BBEF07F00201A0C260
:100920000AF00201FF0E0AB0A56FA561FBEF04F00B
:100930000301A6A1DBEF04F00F0183BEDBEF04F09F
:10094000800E0FEC0DF0000EF86E640EF76E720E56
:10095000F66E75EC0DF0C00E0FEC0DF0000EF86E9B
:10096000640EF76E180EF66E75EC0DF00F01D89050
:1009700084B4D880D8B0C2EF04F00A0E9DEC0BF01E
:100980000F01D89084B4D880D8B0B6EF04F00F012E
:10099000D89084B4D880D8A0C7EF04F00A0E9DEC9C
:1009A0000BF00F01D89084B4D880D8A0C7EF04F022
:1009B000C80E9DEC0BF00201D1B1E2EF04F0D1A31F
:1009C000FBEF04F0800E00019D6F98EC30F0D890A2
:1009D0001EEC27F0D8B0F2EF04F00201FF0EA56F75
:1009E000FBEF04F0E9EC0AF064EC0AF0A1EC0AF089
:1009F0000A0E9DEC0BF00001010E366EA3C252F000
:100A0000A4C253F00201A25100014D6E5AEC23F032
:100A100057EC1FF0FCAE10EF05F00F01939481949A
:100A2000000133B030EF05F0010E366296EF05F0AD
:100A30000001050EE8CF5DF0070E37EC0AF0020E5C
:100A4000366E0001A5510201006329EF05F096EF13
:100A500005F0006FFFEC1EF057EC1FF096EF05F06D
:100A6000010E366EFBEC22F0EDEC17F040EC07F0D7
:100A70000201A1A161EF05F00301B6516FEC24F072
:100A8000D8A061EF05F00201B76759EF05F0ABC0E0
:100A900073F0ACC074F0ADC075F0AEC076F0AFC00E
:100AA00077F0B0C078F0B1C079F0B2C07AF061EF01
:100AB00005F0F08CF086A290E868E8CFEEF067EFE2
:100AC00005F0F09CF086A280E86AE8CFEEF0020123
:100AD000A0B186EF05F01FEC17F0D8B486EF05F053
:100AE000A3EC19F036EC19F070EC1BF002EC1CF0E2
:100AF00001EC1AF090EC21F0AFEC1FF098EC21F033
:100B0000E7EC1AF00001E9672CEC10F062EC03F05E
:100B1000E3EC1CF04EEC0EF00001A26794EF05F040
:100B20000A0EA26FDEEC05F00AEF05F0800E0FEC66
:100B30000DF0000EF86E650EF76EA40EF66E75ECF5
:100B40000DF0C00E0FEC0DF0000EF86E640EF76E97
:100B5000180EF66E75EC0DF073EC1EF0D8A0B3EF26
:100B600005F031EC25F0EDEC17F0A3EC19F036ECC4
:100B700019F070EC1BF002EC1CF001EC1AF090EC98
:100B800021F0AFEC1FF098EC21F0E7EC1AF0E3EC69
:100B90001CF04EEC0EF00AEF05F00001100E0B6E8B
:100BA000C00E0FEC0DF0000EE16E030EE26EE6508B
:100BB00000EC0DF00B2ED7EF05F012000001840EB3
:100BC0000FEC0DF0200E00EC0DF00201520EA5BF4F
:100BD000200E000100EC0DF00601CE516FEC24F068
:100BE000410ED8A0200E00EC0DF00301B2516FECC5
:100BF00024F04D0ED8B02D0E00EC0DF00301B351D2
:100C00006FEC24F04D0ED8B02D0E00EC0DF003016A
:100C1000B4516FEC24F04D0ED8B02D0E00EC0DF059
:100C2000200E00EC0DF0800E0FEC0DF0B9C20DF0AF
:100C3000BAC20EF00E6A0001640E0F6E000E106E46
:100C400057EC10F013C011F014C012F08BC00DF06F
:100C50008CC00EF013C20FF014C210F057EC10F05D
:100C60001450E8CF13F01550E8CF14F0156A0101C5
:100C700011B14BEF06F000011150135C12501458E3
:100C8000E8AE4BEF06F0C90E00015D6E050E37ECC5
:100C90000AF001011169000105EC0EF0200EE8CF09
:100CA0000AF0300E25640AC025F0255000EC0DF046
:100CB000265000EC0DF02E0E00EC0DF0275000EC4D
:100CC0000DF00301B6516FEC24F0D8A071EF06F0DF
:100CD000800E0FEC0DF000C513F001C514F0DBEC35
:100CE0000DF00201B8AF8AEF06F0B86B000EE8CF46
:100CF0000DF0E86AE8CF0EF000C5E8FFB3EC0BF0AA
:100D0000010EE8CF0DF0E86AE8CF0EF001C5E8FF6C
:100D1000B3EC0BF069EC07F0D8B0B4EF06F07AEC66
:100D200007F0D8B0B4EF06F0BCEC24F0D8B0B4EFC4
:100D300006F08EEC23F00001A351E812D8A4B4EF22
:100D400006F00201A0A1B2EF06F0C00E0FEC0DF00C
:100D5000000EF86E640EF76E320EF66E75EC0DF046
:100D6000B4EF06F0CDEC05F0000133B4CFEF06F0A0
:100D700035A4CFEF06F03594010E5D6E050E37EC0D
:100D80000AF000015466CEEF06F0542ABEC358F0B4
:100D9000BFC359F0CA6BCB6BCFEF06F0540600010E
:100DA00054A002EF07F0596602EF07F03B0E5A62BB
:100DB000E1EF06F0050E5D6E0A0E37EC0AF002EF69
:100DC00007F01E0E5A62ECEF06F0030E5D6E0A0E7F
:100DD00037EC0AF002EF07F00A0E5A62F7EF06F05E
:100DE000010E5D6E0A0E37EC0AF002EF07F0060EF8
:100DF0005A6002EF07F0010E5D6E0A0E37EC0AF042
:100E000002EF07F07F0E5A6E5650CE6F5750CF6FDD
:100E1000010E54622BEF07F058505910D8B41AEF56
:100E200007F05850CE6F5950CF6F000E0301BD63CD
:100E30002BEF07F0020E0301BD5DD8B427EF07F0DA
:100E40000001CA51CE6FCB51CF6F2BEF07F0E86A8C
:100E50000001CE6FCF6F00018B0E0FEC0DF0CF5164
:100E6000E8CF13F0146A156A166AD3EC0DF03A0E47
:100E700000EC0DF0CE51E8CF13F0D3EC0DF01200E2
:100E80000301C0516FEC24F0D8A066EF07F0030116
:100E9000000EC16563EF07F000017ABF66EF07F04F
:100EA0000301C15100010D6E0E6A00010A0E0F6EA2
:100EB000000E106E57EC10F07951135E7A51145CED
:100EC000D8B066EF07F00001E76912000001E76B98
:100ED0001200D8900001CCAF1200C00E0FEC0DF044
:100EE000000EF86E640EF76EDE0EF66E75EC0DF009
:100EF000D88012000D0E93EC08F00D0E93EC08F064
:100F000069C00DF06AC00EF0A9C20FF0AAC210F0BD
:100F100057EC10F000011450136E1550146E16505B
:100F2000156E166A05EC0EF00001255026100F0B09
:100F3000D890D8B41200C00E0FEC0DF0000EF86E71
:100F4000640EF76ECC0EF66E75EC0DF0CB0E0FEC5A
:100F50000DF00001255000EC0DF0265000EC0DF0D6
:100F60002E0E00EC0DF0275000EC0DF0285000EC98
:100F70000DF0D88012000F01D89084B4D880D8A08A
:100F8000BBEF07F00A0E9DEC0BF00F01D89084B474
:100F9000D880D8A0BBEF07F00F01D89083B6D880D7
:100FA000D8A0CCEF07F00A0E9DEC0BF00F01D89003
:100FB00083B6D880D8A0CCEF07F0800E0FEC0DF0F0
:100FC0000F01835092EC0DF00F01845092EC0DF064
:100FD000C00E0FEC0DF00F01865092EC0DF00F01DA
:100FE000875092EC0DF00F01835082868184E8B027
:100FF0008296E8B281948098E8B48088320E9DECA5
:101000000BF00F01D89084B4D880D8B00DEF08F061
:101010000A0E9DEC0BF00F01D89084B4D880D8B0A4
:10102000DDEF07F00F01D89084B4D880D8A012EF7C
:1010300008F00A0E9DEC0BF00F01D89084B4D88014
:10104000D8A012EF08F0C00E0FEC0DF0000EF86EF5
:10105000630EF76E880EF66E75EC0DF000010D6AEA
:10106000800E0FEC0DF0000EF86E630EF76EBE0EE4
:10107000F66E75EC0DF0870E0FEC0DF000010D50C3
:101080009FEC0DF093EC08F08C0E0FEC0DF00F01BF
:10109000C4CFE8FF9FEC0DF00F01C3CFE8FF9FEC3A
:1010A0000DF0320E9DEC0BF00F01D89084B4D88077
:1010B000D8B060EF08F00A0E9DEC0BF00F01D8904D
:1010C00084B4D880D8B030EF08F00F01D89084B441
:1010D000D880D8A065EF08F00A0E9DEC0BF00F0148
:1010E000D89084B4D880D8A065EF08F000010D2A0C
:1010F0000C0E0D6430EF08F0DDEF07F00001136A0D
:10110000146A156A166A0A6E0B6A0A5093EC08F0A4
:101110000001C3501326C4501422D8B0152A0B2E38
:1011200085EF08F012000A6EA10EC06E000EC16EAF
:101130000AC0E8FF31EC02F0E8AEC188E89EE8445E
:10114000E844C26EC2800000C282C2B2A5EF08F0BD
:101150000001C3CF69F0C4CF6AF00AC0E8FF1200F3
:101160000F01C282C2B2B2EF08F00001C35069277A
:10117000C4506A23120093EC08F0B0EC08F0B0EC15
:1011800008F0B0EC08F000016A336A9F693312007E
:1011900000014C6A566A576A280EE8CF55F00001E4
:1011A000900E526E010E536E0001900E4E6E010EA7
:1011B0004F6E506A516A100E0001E8CF4DF0386A48
:1011C0003A6A3C6A3E6A406A426A446A466A486AC7
:1011D0004A6A080EE8CF39F0E8CF3BF0E8CF3DF09F
:1011E000E8CF3FF0E8CF41F0E8CF43F0E8CF45F05B
:1011F000E8CF47F0E8CF49F0E8CF4BF0979E858ED7
:10120000000152500F01E8CFBBFF010153500F0105
:10121000E8CFBCFF0A0E0F01E8CFBAFF0F01A08094
:101220000F019E900F01080EE8CFB1FFB1801200B0
:101230000001EEA1857E0201BAAF22EF09F08770AE
:101240002AEF09F00001E5B129EF09F087802AEFC4
:1012500009F087900001BBCFE8FF4E26BCCFE8FF26
:101260004F224EC0E8FFE8CFBBFF4FC0E8FFE8CFFA
:10127000BCFF0001E86A4C64A1EC09F000014C2AB3
:101280004CC0E8FFFE0B4D6057EF09F04C6A500E62
:10129000E8CF4EF050C0E8FF4E5EC30EE8CF4FF0EF
:1012A00051C0E8FF4F5A506A516A9EEF09F04CA0B6
:1012B0006CEF09F052C0E8FFE8CF4EF053C0E8FFF2
:1012C000E8CF4FF0BAC2E8FF0001E5814C6298EF29
:1012D00009F0E59198EF09F0120E4C6284EF09F0E5
:1012E00050C0E8FFE8CF4EF051C0E8FFE8CF4FF024
:1012F0004F324E324F324E324F324E324F324E32EA
:101300000F0E4F1698EF09F0040EE8CFEAFF000E1B
:10131000E8CFE9FF4CC0E8FFE830E89EE804E926A2
:1013200000EC02F052C0E8FF4E5E53C0E8FF4F5A97
:101330004EC0E8FF50264FC0E8FF51220F01A19098
:10134000120083EC0EF08DEC0EF00001010E3662FF
:10135000B0EF09F000018286BDB18296FF0EBD6F2D
:1013600087900301CDBFB8EF09F0859EB9EF09F072
:10137000858E0001552EFFEF09F0BAEC24F0000134
:1013800054A0EFEF09F00001FF0EE763EFEF09F063
:1013900058C0E8FF5910D8B4E7EF09F05866D4EF09
:1013A00009F03C0E586E5906580658505A6E030103
:1013B000E86ABD11D8B4E7EF09F0000158505910A0
:1013C000D8B4E7EF09F0CA6BCB6BEFEF09F000017F
:1013D000CA2B3C0ECA63EFEF09F0CA6BCB2B280E69
:1013E000E8CF55F0562A3C0E5662FFEF09F0566AD8
:1013F000572A0501002BD8B4012B0201B86902015C
:10140000A1A108EF0AF0530EB5EC0EF00001A86B95
:10141000000183CFE8FF311AD8A4306E316E30C09E
:10142000E8FF3212000184CFE8FF341AD8A4336EEB
:10143000346E33C0E8FF351200015E665E065F66FB
:101440005F0660676007A167A107A267A207A3679D
:10145000A3075C662DEF0AF012005C2E1200807864
:101460005D4E12005BC0E8FFE8CF5CF01200E8CFF1
:101470005BF0E8CF5CF08098120000010ABE44EFF8
:101480000AF0819E45EF0AF0818E828A829A0A468E
:101490000B2E3DEF0AF012000201AD510A6E080E4C
:1014A0000B6E3DEC0AF00201AC510A6E080E0B6E99
:1014B0003DEC0AF00201AB510A6E080E0B6E3DECDA
:1014C0000AF08686869612000BC113F00CC114F048
:1014D0000DC115F009C117F00AC118F05BEC11F04D
:1014E0000201A55101010F03F35000011326D8B0EA
:1014F000142AD8B0152A0101006B016B026B0001A0
:101500001350E846E846E880E8921F0B13B6E88ED1
:101510000101006F000113361436153613361436E8
:101520001536133614361536133614361536145050
:101530000101016F000115501F0B01011009026F1D
:10154000120064EC0AF0010108510A6E080E0B6EDD
:101550003DEC0AF0010107510A6E080E0B6E3DECDE
:101560000AF0010106510A6E080E0B6E3DEC0AF0FE
:1015700086868696010105510A6E080E0B6E3DECBB
:101580000AF0010104510A6E080E0B6E3DEC0AF0E0
:10159000010103510A6E080E0B6E3DEC0AF08686BF
:1015A0008696010102510A6E080E0B6E3DEC0AF0A0
:1015B000010101510A6E080E0B6E3DEC0AF00101AB
:1015C00000510A6E080E0B6E3DEC0AF08686869678
:1015D00012000F01939E949A939C819C819E829A03
:1015E000989686960201D1A118EF0BF0D1B318EFAF
:1015F0000BF004C206F105C207F106C208F101C2F0
:1016000003F102C204F103C205F10101700E0B6F78
:10161000C60E0C6F000E0D6F0101140E096F000E47
:101620000A6F01010E6B0A0E106F010E0F6F120090
:101630000201D1B13EEF0BF0D1A33EEF0BF00AC295
:1016400006F10BC207F10CC208F107C203F108C290
:1016500004F109C205F101016C0E0B6FCF0E0C6F86
:10166000000E0D6F0101640E096F000E0A6F01017B
:101670000E6B080E106F010E0F6F12000201D1B138
:1016800065EF0BF0D1B365EF0BF010C206F111C29C
:1016900007F112C208F10DC203F10EC204F10FC22C
:1016A00005F101014A0E0B6F190E0C6F010E0D6F43
:1016B00001010A0E096F000E0A6F01010B0E0E6F79
:1016C000320E106F020E0F6F1200120087B284EFFD
:1016D0000BF0D5AE76EF0BF0D6CFC1F0D7CFC2F07E
:1016E0000001C32BD8B4C42BF09012000001C351E9
:1016F000C411F090D8A41200E86AE8CFD7FFE8CF71
:10170000D6FFD58EF0901200F17AF0AC96EF0BF088
:101710000301CDA192EF0BF0F1AA859EF1BA858E5F
:1017200096EF0BF0F1AA858EF1BA859EF09012002B
:101730000000E82E98EF0BF012000A6EFA0E98ECFB
:101740000BF0FA0E98EC0BF00A2E9EEF0BF0120045
:101750000EC0E8FFAA6E0DC0E8FFA96EA69EA69C6B
:10176000A680A8501200A86E0EC0E8FFAA6E0DC099
:10177000E8FFA96EA69EA69CA684F29E550EA76EB3
:10178000AA0EA76EA682F28EA1A8C4EF0BF0A198B4
:101790001200800E0FEC0DF0000EF86E640EF76E66
:1017A000840EF66E75EC0DF0C00E0FEC0DF0000E11
:1017B000F86E640EF76E060EF66E75EC0DF067ECC3
:1017C00027F0D8A009EF0CF0C00E0FEC0DF0000EC2
:1017D000F86E640EF76E960EF66E75EC0DF081ECF9
:1017E00031F099EC1EF00001600E9E6F00C2E8FF20
:1017F0002AEC1FF00201002B0301072B3A0E0763AE
:1018000005EF0CF0062B300E076F00019E2FF6EF50
:101810000BF084EC1EF000C2E8FFFFEC1EF012009B
:1018200000011550F86E1450F76E1350F66E00015B
:101830000E50E26E0D50E16E0900F550E66E0A069C
:101840000900F550E66E0A2E1CEF0CF012000001A4
:101850001550F86E1450F76E1350F66EA68EA69CB7
:10186000A684A688F29E550EA76EAA0EA76EA68223
:101870000000F28E0001400E1326000E14221522E5
:101880000A2E27EF0CF0120062EC03F00001155055
:10189000F86E1450F76E1350F66EA68EA69CA684B2
:1018A000A688F29E550EA76EAA0EA76EA682F28E8D
:1018B0000A0000010E50E26E0D50E16E400E0B6EFC
:1018C000E6CFE8FFF56E0F000B2EFAD7A68EA69C8A
:1018D000A684F29E550EA76EAA0EA76EA682F28E61
:1018E000A6940001400E1326000E142215220001BA
:1018F000400E0D26000E0E220A2E44EF0CF01200B0
:1019000000011550F86E1450F76E1350F66EA68E47
:10191000A69CA684A688F29E550EA76EAA0EA76E58
:10192000A6820000F28E0A00080E0B6E00010E5017
:10193000E26E0D50E16E080E0C6EE6CFE8FFF56E1C
:101940000F000C2EFAD7A68EA69CA684F29E550EEA
:10195000A76EAA0EA76EA6820000F28E0B2EEBD702
:10196000A6940001400E1326000E14221522000139
:10197000400E0D26000E0E220A2E80EF0CF01200F3
:101980000F019A6A886A9396939A93988186818ABE
:101990008188140E9DEC0BF0380E0FEC0DF0050E47
:1019A0009DEC0BF0380E0FEC0DF0010E9DEC0BF0E2
:1019B000380E0FEC0DF0010E9DEC0BF0380E0FEC15
:1019C0000DF0060E0FEC0DF00E0E0FEC0DF0010EEB
:1019D0000FEC0DF0800E0FEC0DF0800E0FEC0DF003
:1019E000630EF76E9A0EF66E75EC0DF0C00E0FECEE
:1019F0000DF0630EF76EAC0EF66E75EC0DF0120086
:101A00001EEC0DF032EC0DF0818A81980000000090
:101A100081860000000081960000000012001EEC8C
:101A20000DF032EC0DF0819A819800000000818663
:101A300000000000819600000000120025EC0DF06F
:101A4000D8B01EEF0DF09A6A12009A688188819AC8
:101A500000000000818600000000D89088BED88079
:101A600081961200886E12001010101010101010C5
:101A700018181818181818181C1C1C1C1C1C1C1CC6
:101A80001E1E1E1E1E1E1E1E01010101010101015E
:101A900003030303030303030707070707070707F6
:101AA0000F0F0F0F0F0F0F0F800E0FEC0DF00DC06B
:101AB000F6FF0EC0F7FFF86A75EC0DF01200C00ECD
:101AC0000FEC0DF00DC0F6FF0EC0F7FFF86A75ECD5
:101AD0000DF01200C00E0FEC0DF0CEC0F6FFCFC01F
:101AE000F7FFF86A75EC0DF01200100E78EF0DF0AC
:101AF0000A6E0900F5CFE8FFE812D8B491EF0DF0B7
:101B000000EC0DF00A4E91EF0DF00900F5CFE8FF63
:101B1000E812D8B491EF0DF000EC0DF00A2E79EF39
:101B20000DF012000A6E080E0B6E300E0ABE310E5A
:101B300000EC0DF00A360B2E95EF0DF012000A6E38
:101B40003A0E0B6E0AC0E8FFF00BE842E842E842AA
:101B5000E84230090B64070F00EC0DF00AC0E8FF03
:101B60000F0B30090B64070F00EC0DF00AC0E8FF03
:101B7000120005EC0EF0255000EC0DF0265000ECA4
:101B80000DF0275000EC0DF0285000EC0DF029501E
:101B900000EC0DF0120005EC0EF0BEEF0DF005ECC0
:101BA0000EF0C1EF0DF005EC0EF0C4EF0DF005ECFA
:101BB0000EF0C7EF0DF005EC0EF0EFEC0DF0255038
:101BC00000EC0DF0265000EC0DF0275000EC0DF06D
:101BD000285000EC0DF0295000EC0DF0120000012F
:101BE000300E25621200200E256E300E2662120085
:101BF000200E266E300E27621200200E276E300E49
:101C000028621200200E286E12000001196A1A6A5A
:101C1000100E176E270E186E5BEC11F0300E1310BD
:101C2000256E1BC013F01CC014F01DC015F01EC0A3
:101C300016F0196A1A6AE80E176E030E186E5BEC3E
:101C400011F0300E1310266E1BC013F01CC014F0E0
:101C50001DC015F01EC016F0196A1A6A640E176EC0
:101C6000000E186E5BEC11F0300E1310276E1BC0C7
:101C700013F01CC014F01DC015F01EC016F0196A38
:101C80001A6A0A0E176E000E186E5BEC11F0300E19
:101C90001310286E300E1B10296E12000001310E39
:101CA000376257EF0EF084EC1EF081EF0EF0320E2B
:101CB000376261EF0EF000C2E8FFFFEC1EF081EF2B
:101CC0000EF0330E376269EF0EF099EC1EF081EFE3
:101CD0000EF0340E376271EF0EF000C2E8FF2AEC0E
:101CE0001FF0350E376281EF0EF00001FF0E0D6E12
:101CF000030E0E6EE8CF0EF0FF0EB3EC0BF081EF8B
:101D00000EF0376A12000F01ABA21200AB98AB883D
:101D10000F01AE500001616B12000F016BA21200A7
:101D20006B986B880F016E5012000C0EE8CFAFFF5E
:101D3000220EE8CFACFF900EE8CFABFF0001616B45
:101D40009F9A9D8A1200ACA2A3EF0EF0E8CFADFFE0
:101D50001200000EE8CF6FFF220EE8CF6CFF900E4E
:101D6000E8CF6BFFA59AA38A12006CA2B5EF0EF024
:101D7000E8CF6DFF1200E1CF21F0E2CF22F00001A9
:101D800065C0E1FF000164C0E2FF686BACA2C6EF72
:101D90000EF0E6CFE8FF00016827E8CFADFF0001B5
:101DA000662FC6EF0EF021C0E1FF22C0E2FF120055
:101DB000E1CF21F0E2CF22F0000165C0E1FF000198
:101DC00064C0E2FF686B0001050E5E6EE86A5E6447
:101DD000F7EF0EF09EAAE7EF0EF0AECFE8FFE8CFE8
:101DE000E6FF000168270001662FE3EF0EF021C037
:101DF000E1FF22C0E2FF12009EAA12000001000EC5
:101E000061630FEF0FF0AECFE8FFE8CF62F0550E41
:101E100062631200280EE8CF5FF0612B1200010E02
:101E2000616319EF0FF0AECFE8FFE8CF63F0612BED
:101E30001200020E616323EF0FF0AECFE8FFE8CF90
:101E400064F0612B1200030E61632DEF0FF0AECF33
:101E5000E8FFE8CF65F0612B1200040E616336EFF6
:101E60000FF0AECFE8FFE8CF66F0612B050E61639F
:101E700042EF0FF0010E636340EF0FF0D8EC0EF06D
:101E8000612B1200060E616365EF0FF0AECFE8FF25
:101E9000E8CF67F0020E636356EF0FF0BBEC0EF075
:101EA00068C0E8FFA3EC0EF0616B120068C0E8FFA9
:101EB000676360EF0FF00C0EA3EC0EF0616B120085
:101EC0000D0EA3EC0EF0616B1200616B1200A4AA60
:101ED00012006ECFE8FF0201A1B19BEF0FF0530A91
:101EE000D8A412000201A0A1120000010F0E741567
:101EF0001009B5EC0EF073C0E8FFB5EC0EF0000170
:101F00000F0E76152009B5EC0EF07551B5EC0EF0FC
:101F100000010F0E78153009B5EC0EF07751B5ECD5
:101F20000EF000010F0E7A154009B5EC0EF0795154
:101F3000B5EC0EF012000001A8B1A2EF0FF0AA6FED
:101F4000A82B1200A96FA82B020EA863BBEF0FF0FD
:101F5000AA51F00B100AD8A400EF10F00F0EAA1728
:101F6000AAA7B5EF0FF0F00EAA13A9C0ABF0AAC054
:101F7000ACF000EF10F0040EA863D2EF0FF0AA51FE
:101F8000F00B200AD8A400EF10F00F0EAA17AAA792
:101F9000CCEF0FF0F00EAA13A9C0ADF0AAC0AEF0BE
:101FA00000EF10F0060EA863E9EF0FF0AA51F00B56
:101FB000300AD8A400EF10F00F0EAA17AAA7E3EF7B
:101FC0000FF0F00EAA13A9C0AFF0AAC0B0F000EF56
:101FD00010F0080EA86300EF10F0AA51F00B400AB1
:101FE000D8A400EF10F00F0EAA17AAA7FAEF0FF06F
:101FF000F00EAA13A9C0B1F0AAC0B2F000EF10F021
:1020000012000C0E0F016F6E220E6C6E900EE8CF58
:102010006BFF12000001E80E0D26030E0E22780E53
:102020000D5C070E0E58D8A019EF10F0EF0E20EF40
:1020300010F00E320D320E320D320E320D320D50C6
:10204000B5EF0EF0BC0E0D5C030E0E58D8A01BEFC2
:1020500010F0EF0E20EF10F0F00EB5EC0EF0800E49
:10206000B5EC0EF073C00DF074C00EF00AEC10F079
:1020700075C00DF076C00EF00AEC10F077C00DF0D0
:1020800078C00EF00AEC10F079C00DF07AC00EF0B6
:1020900022EC10F07BC00DF07CC00EF022EC10F0B2
:1020A0007DC00DF07EC00EF022EC10F0120068EC46
:1020B00010F010AE60EF10F00D50155E0E50165A75
:1020C0000EAE67EF10F00F50155E1050165A12004A
:1020D0000001136A146A156A166A0F500D02F3CFD5
:1020E00013F0F4CF14F00F500E02F3501426F450F6
:1020F0001522D8B0162A10500D02F3501426F450B1
:102100001522D8B0162A10500E02F3501526F4509E
:10211000162212000001246A1B6A14501310D8B44E
:10212000000C14501718E8BE241EA46B000E17AE46
:102130009CEF10F0171E172A14AEA3EF10F0131E19
:10214000141E132A142214501710E8BE2FEF11F09A
:1021500017501B5E143614341B3617501B261436CA
:1021600014341B36175014B01B5E14A01B261436F3
:1021700014341B36175014B01B5E14A01B261436E3
:1021800014341B36175014B01B5E14A01B261436D3
:1021900014341B36175014B01B5E14A01B261436C3
:1021A00014341B36175014B01B5E14A01B261436B3
:1021B00014341B36175014B01B5E14A01B261436A3
:1021C00013341B36175014B01B5E14A01B26133695
:1021D00013341B36175013B01B5E13A01B26133687
:1021E00013341B36175013B01B5E13A01B26133677
:1021F00013341B36175013B01B5E13A01B26133667
:1022000013341B36175013B01B5E13A01B26133656
:1022100013341B36175013B01B5E13A01B26133646
:1022200013341B36175013B01B5E13A01B26133636
:1022300013341B36175013B01B5E13A01B26133626
:1022400013A01B26A4B14DEF11F024AE000C131EF9
:10225000141EE86A132A14221B1E1B2A000C17AE38
:1022600048EF11F014BE44EF11F0E8CF9DF0135089
:10227000E8CF1BF01B9E133614361450E8CF13F032
:102280009D51146A25EF11F0136A132A146A000C89
:10229000141E131EA42BA8EF10F01B2A17501B624C
:1022A00025EF11F01B6A000E132A142214AE25EF3D
:1022B00011F02388FF0C0001246A1C6A1B6A155068
:1022C00014101310D8B4000C15501818E8BE241EB2
:1022D000A46B000E18AE71EF11F0171E181E172A0E
:1022E000182215AE7AEF11F0131E141E151E132AB4
:1022F0001422152215501810E8BE04EF13F01750E1
:102300001B5E18501C5A153615341B361C361750D8
:102310001B2618501C22153615341B361C36175038
:1023200015A098EF11F01B5E18501C5A9BEF11F08E
:102330001B2618501C22153615341B361C36175018
:1023400015A0A8EF11F01B5E18501C5AABEF11F04E
:102350001B2618501C22153615341B361C361750F8
:1023600015A0B8EF11F01B5E18501C5ABBEF11F00E
:102370001B2618501C22153615341B361C361750D8
:1023800015A0C8EF11F01B5E18501C5ACBEF11F0CE
:102390001B2618501C22153615341B361C361750B8
:1023A00015A0D8EF11F01B5E18501C5ADBEF11F08E
:1023B0001B2618501C22153615341B361C36175098
:1023C00015A0E8EF11F01B5E18501C5AEBEF11F04E
:1023D0001B2618501C22153614341B361C36175079
:1023E00015A0F8EF11F01B5E18501C5AFBEF11F00E
:1023F0001B2618501C22143614341B361C3617505A
:1024000014A008EF12F01B5E18501C5A0BEF12F0CC
:102410001B2618501C22143614341B361C36175039
:1024200014A018EF12F01B5E18501C5A1BEF12F08C
:102430001B2618501C22143614341B361C36175019
:1024400014A028EF12F01B5E18501C5A2BEF12F04C
:102450001B2618501C22143614341B361C361750F9
:1024600014A038EF12F01B5E18501C5A3BEF12F00C
:102470001B2618501C22143614341B361C361750D9
:1024800014A048EF12F01B5E18501C5A4BEF12F0CC
:102490001B2618501C22143614341B361C361750B9
:1024A00014A058EF12F01B5E18501C5A5BEF12F08C
:1024B0001B2618501C22143614341B361C36175099
:1024C00014A068EF12F01B5E18501C5A6BEF12F04C
:1024D0001B2618501C22143613341B361C3617507A
:1024E00014A078EF12F01B5E18501C5A7BEF12F00C
:1024F0001B2618501C22133613341B361C3617505B
:1025000013A088EF12F01B5E18501C5A8BEF12F0CC
:102510001B2618501C22133613341B361C3617503A
:1025200013A098EF12F01B5E18501C5A9BEF12F08C
:102530001B2618501C22133613341B361C3617501A
:1025400013A0A8EF12F01B5E18501C5AABEF12F04C
:102550001B2618501C22133613341B361C361750FA
:1025600013A0B8EF12F01B5E18501C5ABBEF12F00C
:102570001B2618501C22133613341B361C361750DA
:1025800013A0C8EF12F01B5E18501C5ACBEF12F0CC
:102590001B2618501C22133613341B361C361750BA
:1025A00013A0D8EF12F01B5E18501C5ADBEF12F08C
:1025B0001B2618501C22133613341B361C3617509A
:1025C00013A0E8EF12F01B5E18501C5AEBEF12F04C
:1025D0001B2618501C22133613B0F3EF12F01750BD
:1025E0001B2618501C22A4B128EF13F024AE000CB7
:1025F000131E141E151E000E132A142215221B1E54
:102600001C1E1B2A1C22000C18AE22EF13F015BE54
:102610001DEF13F0E8CF9DF01450E8CF1CF01350DD
:10262000E8CF1BF01C9E143615361550E8CF13F07A
:102630009D51156A146AF6EF12F0136A132A146A90
:10264000156A000C151E141E131EA42B7FEF11F02B
:102650001B2AE86A1C2217501B62F6EF12F0185072
:102660001C62F6EF12F01C6A1B6A000E132A142279
:10267000152215AEF6EF12F02388FF0C1E6A1D6AB4
:102680001C6A1B6A16341B361C361D361E36175044
:102690001B5E18501C5A19501D5A1A501E5AA46A13
:1026A000A45B163616341B361C361D361E36A43770
:1026B000175016A067EF13F01B5E18501C5A1950E4
:1026C0001D5A1A501E5AE86AA45B70EF13F01B26BD
:1026D00018501C2219501D221A501E22E86AA423E9
:1026E000163616341B361C361D361E36A4371750C8
:1026F00016A086EF13F01B5E18501C5A19501D5A75
:102700001A501E5AE86AA45B8FEF13F01B2618506C
:102710001C2219501D221A501E22E86AA4231636C4
:1027200016341B361C361D361E36A437175016A01D
:10273000A5EF13F01B5E18501C5A19501D5A1A5061
:102740001E5AE86AA45BAEEF13F01B2618501C2239
:1027500019501D221A501E22E86AA4231636163478
:102760001B361C361D361E36A437175016A0C4EF74
:1027700013F01B5E18501C5A19501D5A1A501E5A3D
:10278000E86AA45BCDEF13F01B2618501C221950E9
:102790001D221A501E22E86AA423163616341B3650
:1027A0001C361D361E36A437175016A0E3EF13F063
:1027B0001B5E18501C5A19501D5A1A501E5AE86AAE
:1027C000A45BECEF13F01B2618501C2219501D229D
:1027D0001A501E22E86AA423163616341B361C36FD
:1027E0001D361E36A437175016A002EF14F01B5EDC
:1027F00018501C5A19501D5A1A501E5AE86AA45BE8
:102800000BEF14F01B2618501C2219501D221A50D1
:102810001E22E86AA423163616341B361C361D36D3
:102820001E36A437175016A021EF14F01B5E185067
:102830001C5A19501D5A1A501E5AE86AA45B2AEFF6
:1028400014F01B2618501C2219501D221A501E224B
:10285000E86AA423163615341B361C361D361E3680
:10286000A437175016A040EF14F01B5E18501C5AE6
:1028700019501D5A1A501E5AE86AA45B49EF14F009
:102880001B2618501C2219501D221A501E22E86ABD
:10289000A423153615341B361C361D361E36A437B8
:1028A000175015A05FEF14F01B5E18501C5A1950FA
:1028B0001D5A1A501E5AE86AA45B68EF14F01B26D2
:1028C00018501C2219501D221A501E22E86AA423F7
:1028D000153615341B361C361D361E36A4371750D8
:1028E00015A07EEF14F01B5E18501C5A19501D5A8B
:1028F0001A501E5AE86AA45B87EF14F01B26185082
:102900001C2219501D221A501E22E86AA4231536D3
:1029100015341B361C361D361E36A437175015A02D
:102920009DEF14F01B5E18501C5A19501D5A1A5076
:102930001E5AE86AA45BA6EF14F01B2618501C224E
:1029400019501D221A501E22E86AA4231536153488
:102950001B361C361D361E36A437175015A0BCEF8B
:1029600014F01B5E18501C5A19501D5A1A501E5A4A
:10297000E86AA45BC5EF14F01B2618501C221950FE
:102980001D221A501E22E86AA423153615341B3660
:102990001C361D361E36A437175015A0DBEF14F079
:1029A0001B5E18501C5A19501D5A1A501E5AE86ABC
:1029B000A45BE4EF14F01B2618501C2219501D22B2
:1029C0001A501E22E86AA423153615341B361C360D
:1029D0001D361E36A437175015A0FAEF14F01B5EF3
:1029E00018501C5A19501D5A1A501E5AE86AA45BF6
:1029F00003EF15F01B2618501C2219501D221A50E7
:102A00001E22E86AA423153615341B361C361D36E3
:102A10001E36A437175015A019EF15F01B5E18507D
:102A20001C5A19501D5A1A501E5AE86AA45B22EF0C
:102A300015F01B2618501C2219501D221A501E2258
:102A4000E86AA423153614341B361C361D361E3690
:102A5000A437175015A038EF15F01B5E18501C5AFC
:102A600019501D5A1A501E5AE86AA45B41EF15F01E
:102A70001B2618501C2219501D221A501E22E86ACB
:102A8000A423143614341B361C361D361E36A437C8
:102A9000175014A057EF15F01B5E18501C5A195010
:102AA0001D5A1A501E5AE86AA45B60EF15F01B26E7
:102AB00018501C2219501D221A501E22E86AA42305
:102AC000143614341B361C361D361E36A4371750E8
:102AD00014A076EF15F01B5E18501C5A19501D5AA1
:102AE0001A501E5AE86AA45B7FEF15F01B26185097
:102AF0001C2219501D221A501E22E86AA4231436E3
:102B000014341B361C361D361E36A437175014A03D
:102B100095EF15F01B5E18501C5A19501D5A1A508B
:102B20001E5AE86AA45B9EEF15F01B2618501C2263
:102B300019501D221A501E22E86AA4231436143498
:102B40001B361C361D361E36A437175014A0B4EFA2
:102B500015F01B5E18501C5A19501D5A1A501E5A57
:102B6000E86AA45BBDEF15F01B2618501C22195013
:102B70001D221A501E22E86AA423143614341B3670
:102B80001C361D361E36A437175014A0D3EF15F08F
:102B90001B5E18501C5A19501D5A1A501E5AE86ACA
:102BA000A45BDCEF15F01B2618501C2219501D22C7
:102BB0001A501E22E86AA423143614341B361C361D
:102BC0001D361E36A437175014A0F2EF15F01B5E09
:102BD00018501C5A19501D5A1A501E5AE86AA45B04
:102BE000FBEF15F01B2618501C2219501D221A50FD
:102BF0001E22E86AA423143614341B361C361D36F4
:102C00001E36A437175014A011EF16F01B5E185093
:102C10001C5A19501D5A1A501E5AE86AA45B1AEF22
:102C200016F01B2618501C2219501D221A501E2265
:102C3000E86AA423143613341B361C361D361E36A0
:102C4000A437175014A030EF16F01B5E18501C5A12
:102C500019501D5A1A501E5AE86AA45B39EF16F033
:102C60001B2618501C2219501D221A501E22E86AD9
:102C7000A423133613341B361C361D361E36A437D8
:102C8000175013A04FEF16F01B5E18501C5A195026
:102C90001D5A1A501E5AE86AA45B58EF16F01B26FC
:102CA00018501C2219501D221A501E22E86AA42313
:102CB000133613341B361C361D361E36A4371750F8
:102CC00013A06EEF16F01B5E18501C5A19501D5AB7
:102CD0001A501E5AE86AA45B77EF16F01B261850AC
:102CE0001C2219501D221A501E22E86AA4231336F2
:102CF00013341B361C361D361E36A437175013A04E
:102D00008DEF16F01B5E18501C5A19501D5A1A50A0
:102D10001E5AE86AA45B96EF16F01B2618501C2278
:102D200019501D221A501E22E86AA42313361334A8
:102D30001B361C361D361E36A437175013A0ACEFB9
:102D400016F01B5E18501C5A19501D5A1A501E5A64
:102D5000E86AA45BB5EF16F01B2618501C22195028
:102D60001D221A501E22E86AA423133613341B3680
:102D70001C361D361E36A437175013A0CBEF16F0A5
:102D80001B5E18501C5A19501D5A1A501E5AE86AD8
:102D9000A45BD4EF16F01B2618501C2219501D22DC
:102DA0001A501E22E86AA423133613341B361C362D
:102DB0001D361E36A437175013A0EAEF16F01B5E1F
:102DC00018501C5A19501D5A1A501E5AE86AA45B12
:102DD000F3EF16F01B2618501C2219501D221A5012
:102DE0001E22E86AA423133613341B361C361D3604
:102DF0001E36A437175013A009EF17F01B5E1850AA
:102E00001C5A19501D5A1A501E5AE86AA45B12EF38
:102E100017F01B2618501C2219501D221A501E2272
:102E2000E86AA423133613B01EEF17F017501B26C1
:102E300018501C2219501D221A501E22000C0F017E
:102E4000D89083B6D880D8B02BEF17F00A0E9DEC3F
:102E50000BF00F01D89083B6D880D8B0A1EF17F04F
:102E60000F01D89084B2D880D8B03CEF17F00A0E8A
:102E70009DEC0BF00F01D89084B2D880D8B0A1EFB0
:102E800017F00001CC6763EF17F00001CC69030174
:102E900032C30DF033C30EF00001E80E0F6E030EC7
:102EA000106E57EC10F014C01CF115C01DF1030199
:102EB000345101011C270301355101011D2334C385
:102EC0001AF135C31BF198EC29F0D8B074EF17F064
:102ED000D8A47BEF17F001011A07D8A01B071A0727
:102EE000D8A01B077BEF17F001011A2BD8B41B2BBE
:102EF0001A2BD8B41B2B1CC10DF01DC10EF0010103
:102F00001A5100010D5E01011B5100010E5A000112
:102F1000000E0F6E010E106E57EC10F00001E80E5F
:102F2000176E030E186E5BEC11F013C032F314C071
:102F300033F31AC134F31BC135F301EC1AF0D88412
:102F400012000001CC67A7EF17F0D8941200CC6BE9
:102F500074EC1FF0D894120000016951E8CF0DF015
:102F60006A51E8CF0EF06D510D5E6E510E5AD8A029
:102F7000C9EF17F06B51E8CF0FF06C51E8CF10F0AC
:102F800057EC10F01450E8CF71F01550E8CF72F004
:102F900012006F51E8CF0FF07051E8CF10F057ECEE
:102FA00010F01450E8CF71F01550E8CF72F0120015
:102FB00069C00DF06AC00EF06D510D5E6E510E5A73
:102FC0006BC00FF06CC010F057EC10F01450E8CF4D
:102FD00071F01550E8CF72F01200040E93EC08F077
:102FE000040EBBEC08F015C26BF016C26CF017C2F1
:102FF0006DF018C26EF019C26FF01AC270F0ACEC2E
:1030000017F071C034F172C035F171C073F072C045
:1030100074F0050E93EC08F0050EBBEC08F01BC233
:103020006BF01CC26CF01DC26DF01EC26EF01FC2B0
:103030006FF020C270F0ACEC17F071C036F172C0C6
:1030400037F171C075F072C076F0060E93EC08F09F
:10305000060EBBEC08F021C26BF022C26CF023C25A
:103060006DF024C26EF025C26FF026C270F0ACEC99
:1030700017F071C038F172C039F171C077F072C0C9
:1030800078F0070E93EC08F0070E93EC08F027C2D7
:103090006BF028C26CF029C26DF02AC26EF0D8EC39
:1030A00017F071C03AF172C03BF171C079F072C093
:1030B0007AF0030E93EC08F000010F01C3CFE8FF94
:1030C000E8CF8BF0C4CFE8FFE8CF8CF0080E93EC8C
:1030D00008F02DC26DF02EC26EF02BC26BF02CC228
:1030E0006CF0D8EC17F071C083F072C084F0090E58
:1030F00093EC08F031C26DF032C26EF02FC26BF06B
:1031000030C26CF0D8EC17F071C085F072C086F058
:103110000A0E93EC08F035C26DF036C26EF033C281
:103120006BF034C26CF0D8EC17F071C087F072C04D
:1031300088F00B0E93EC08F039C26DF03AC26EF0D5
:1031400037C26BF038C26CF0D8EC17F071C089F060
:1031500072C08AF00301B5516FEC24F0D8A0B7EF2C
:1031600018F0030E7C6FE80E7B6FB9EF18F07B6BE5
:103170007C6B000E93EC08F03BC26BF03CC26CF031
:103180003DC26DF03EC26EF0D8EC17F071C07DF01C
:1031900072C07EF0010E93EC08F03FC26BF040C2AB
:1031A0006CF041C26DF042C26EF0D8EC17F071C005
:1031B0007FF072C080F00301B7516FEC24F0D8A00B
:1031C000E8EF18F0030E826FE80E816FFEEF18F043
:1031D0000301B9516FEC24F0D8A0F3EF18F0816B24
:1031E000826BFEEF18F00301B8516FEC24F0D8A009
:1031F000FEEF18F0010E826FF40E816F12000001D5
:10320000106A0FBE101E57EC10F00001640E176E0E
:10321000000E186E5BEC11F013C011F014C012F028
:1032200013C00FF014C010F00EAE1CEF19F00F1EFB
:10323000101E0F2AD8B0102A57EC10F000010A0E09
:10324000176E000E186E5BEC11F00B50E8CF17F004
:10325000186A17BE181E5BEC11F011500D5E12506B
:103260000E5A13500D2614500E2212000301AE51B7
:103270006FEC24F073C00DF074C00EF0D8A04CEFCA
:1032800019F003011B510001E8CF0FF003011751A2
:10329000E8CF0BF054EF19F003011A510001E8CF09
:1032A0000FF0640EE8CF0BF0FFEC18F00DC073F0D8
:1032B0000EC074F00301AF516FEC24F075C00DF037
:1032C00076C00EF0D8A070EF19F00301265100016E
:1032D000E8CF0FF003012251E8CF0BF078EF19F09F
:1032E000030125510001E8CF0FF0640EE8CF0BF089
:1032F000FFEC18F00DC075F00EC076F00301B05170
:103300006FEC24F077C00DF078C00EF0D8A094EFE9
:1033100019F0030131510001E8CF0FF003012D51E5
:10332000E8CF0BF09CEF19F0030130510001E8CF1A
:103330000FF0640EE8CF0BF0FFEC18F00DC077F043
:103340000EC078F012000301AE516FEC24F0D8A04B
:10335000C2EF19F073C00FF074C010F017C30DF076
:1033600018C30EF00E6A0DBE0E1E57EC10F00001D1
:10337000640E176E000E186E5BEC11F013C073F044
:1033800014C074F00301AF516FEC24F0D8A0E1EF4A
:1033900019F075C00FF076C010F022C30DF023C3F2
:1033A0000EF00E6A0DBE0E1E57EC10F00001640EFA
:1033B000176E000E186E5BEC11F013C075F014C0A0
:1033C00076F00301B0516FEC24F0D8A000EF1AF0B2
:1033D00077C00FF078C010F02DC30DF02EC30EF0A3
:1033E0000E6A0DBE0E1E57EC10F00001640E176E33
:1033F000000E186E5BEC11F013C077F014C078F07B
:1034000012000201B2519BEC01F00301A75100012F
:103410000F260301A8510001102218C30DF019C393
:103420000EF000010E6AFF0E0DBE0E6E57EC10F08E
:103430000001640E176E186A196A1A6A5BEC11F0C3
:1034400000010301195100010D6E0E6A0DBE0E1E22
:103450000D360E360D5013260E50142213507327BE
:10346000145074230201B3519BEC01F00301A951E4
:1034700000010F260301AA510001102223C30DF001
:1034800024C30EF000010E6AFF0E0DBE0E6E57EC47
:1034900010F00001640E176E186A196A1A6A5BEC64
:1034A00011F000010301245100010D6E0E6A0DBEE2
:1034B0000E1E0D360E360D5013260E5014221350CC
:1034C0007527145076230201B4519BEC01F00301DF
:1034D000AB5100010F260301AC51000110222EC395
:1034E0000DF02FC30EF000010E6AFF0E0DBE0E6E22
:1034F00057EC10F00001640E176E186A196A1A6A08
:103500005BEC11F0000103012F5100010D6E0E6AFA
:103510000DBE0E1E0D360E360D5013260E50142203
:1035200013507727145078230201B5519BEC01F01A
:1035300036C30DF037C30EF000010E6AFF0E0DBE4C
:103540000E6E57EC10F00001640E176E186A196ABF
:103550001A6A5BEC11F00301010E3763C7EF1AF032
:103560000001030E0E6E186EE80E0D6E176E795187
:103570000D5E7A510E5A196A1A6A13C00FF014C000
:1035800010F057EC10F05BEC11F0E1EF1AF0020EC6
:103590003763E1EF1AF0000179510D6E7A510E6E2A
:1035A00013C00FF014C010F057EC10F00001030E20
:1035B000E8CF18F0E80EE8CF17F0196A1A6A5BEC4A
:1035C00011F000011350792714507A2312000001E2
:1035D0000E6A08C40DF00DBE0E6800010A0E0F6ED3
:1035E000000E106E57EC10F0135073271450742314
:1035F00000010E6A09C40DF00DBE0E6800010A0E2E
:103600000F6E000E106E57EC10F01350752714500B
:10361000762300010E6A0AC40DF00DBE0E6800018B
:103620000A0E0F6E000E106E57EC10F01350772735
:103630001450782300010E6A0BC40DF00DBE0E6805
:1036400000010A0E0F6E000E106E57EC10F01350B2
:10365000792714507A2300010E6A0CC40DF00DBEB8
:103660000E6800010A0E0F6E000E106E57EC10F07F
:1036700013507B2714507C2300010E6A0DC40DF0FB
:103680000DBE0E6800010A0E0F6E000E106E57EC94
:1036900010F013507D2714507E2300010E6A0EC4D3
:1036A0000DF00DBE0E6800010A0E0F6E000E106EBA
:1036B00057EC10F013507F271450802300010E6A3E
:1036C0000FC40DF00DBE0E6800010A0E0F6E000E45
:1036D000106E57EC10F01350812714508223120003
:1036E00000010A0E0D6E000E0E6E0301BB516FEC51
:1036F00024F0D8A0B8EF1BF003014DAF8BEF1BF007
:103700004CC30FF0106A0FBE106857EC10F013C0D6
:1037100073F014C074F003014FAF9AEF1BF04EC367
:103720000FF0106A0FBE106857EC10F013C075F060
:1037300014C076F0030151AFA9EF1BF050C30FF096
:10374000106A0FBE106857EC10F013C077F014C069
:1037500078F0030153AFB8EF1BF052C30FF0106ABB
:103760000FBE106857EC10F013C079F014C07AF057
:103770000301BC516FEC24F0D8A0FBEF1BF0030158
:1037800055AFCEEF1BF054C30FF0106A0FBE106898
:1037900057EC10F013C073F014C074F0030157AF6E
:1037A000DDEF1BF056C30FF0106A0FBE106857EC28
:1037B00010F013C075F014C076F0030159AFECEFB0
:1037C0001BF058C30FF0106A0FBE106857EC10F0D2
:1037D00013C077F014C078F003015BAFFBEF1BF070
:1037E0005AC30FF0106A0FBE106857EC10F013C0E8
:1037F00079F014C07AF000017AAF1200E86A796FAC
:103800007A6F12000201A1B112000301B6516FECF0
:1038100024F0D8A0120000016067120002019F513D
:103820000001606F0201010EB66320EF1CF0010E73
:1038300000015D6E050E37EC0AF0280E0001606F86
:1038400073C00DF074C00EF0C3EC1CF0D8A456EF9A
:103850001CF00201B6672FEF1CF002019E5100011F
:1038600074BF3DEF1CF00301192719AF47EF1CF09F
:10387000D8A647EF1CF04AEF1CF00301195F19BFEF
:1038800047EF1CF0D8A647EF1CF04FEF1CF019BF14
:103890004FEF1CF0640E1961196F54EF1CF0640EA9
:1038A000E81EE82A1965196F74EC1FF075C00DF059
:1038B00076C00EF0C3EC1CF0D8A48CEF1CF0020113
:1038C000B66765EF1CF002019E51000176BF73EFF1
:1038D0001CF00301242724AF7DEF1CF0D8A67DEF58
:1038E0001CF080EF1CF00301245F24BF7DEF1CF06F
:1038F000D8A67DEF1CF085EF1CF024BF85EF1CF0EF
:10390000640E2461246F8AEF1CF0640EE81EE82A1E
:103910002465246F74EC1FF077C00DF078C00EF0B2
:10392000C3EC1CF0D8A4C2EF1CF00201B6679BEFF9
:103930001CF002019E51000178BFA9EF1CF00301A9
:103940002F272FAFB3EF1CF0D8A6B3EF1CF0B6EFC4
:103950001CF003012F5F2FBFB3EF1CF0D8A6B3EF0D
:103960001CF0BBEF1CF02FBFBBEF1CF0640E2F61EF
:103970002F6FC0EF1CF0640EE81EE82A2F652F6F32
:1039800074EC1FF0120000010EAECCEF1CF00D1E07
:103990000E1E0D2AD8B00E2AD8900E320D320E66A9
:1039A000D6EF1CF0640E0D64DBEF1CF00001640E1A
:1039B0000D6E000E0E6E0D50E832E8321F0BD874FB
:1039C0000DC0E8FF12000001BD6B000174BFF5EFF0
:1039D0001CF011C30DF012C30EF073C00FF074C0D1
:1039E00010F057EC10F0FFEF1CF015C30DF016C3EC
:1039F0000EF073C00FF074C010F057EC10F013C34A
:103A00000DF014C30EF0000114500D2615500E22B7
:103A100054EC1EF00DC03CF00EC03DF0000176BF2E
:103A20001EEF1DF01CC30DF01DC30EF075C00FF08E
:103A300076C010F057EC10F028EF1DF020C30DF009
:103A400021C30EF075C00FF076C010F057EC10F0E7
:103A50001EC30DF01FC30EF0000114500D261550AB
:103A60000E2254EC1EF00DC03AF00EC03BF00001E7
:103A700078BF47EF1DF027C30DF028C30EF077C0C5
:103A80000FF078C010F057EC10F051EF1DF02BC381
:103A90000DF02CC30EF077C00FF078C010F057EC8B
:103AA00010F029C30DF02AC30EF0000114500D26AA
:103AB00015500E2254EC1EF00DC03EF00EC03FF02B
:103AC00032C30DF033C30EF079C00FF07AC010F09E
:103AD00057EC10F034C30DF035C30EF00001145054
:103AE0000D2615500E2254EC1EF00DC040F00EC0F5
:103AF00041F03AC30DF03BC30EF07BC00FF07CC029
:103B000010F057EC10F03CC30DF03DC30EF0000177
:103B100014500D2615500E2254EC1EF00DC042F02C
:103B20000EC043F0040117A1BBEF1DF000017EBFE2
:103B3000A6EF1DF01CC30DF01DC30EF07DC00FF0ED
:103B40007EC010F057EC10F0B0EF1DF020C30DF068
:103B500021C30EF07DC00FF07EC010F057EC10F0C6
:103B60001EC30DF01FC30EF0000114500D2615509A
:103B70000E22CEEF1DF03EC30DF03FC30EF07DC010
:103B80000FF07EC010F057EC10F040C30DF041C3B1
:103B90000EF0000114500D2615500E2254EC1EF0AC
:103BA0000DC044F00EC045F003019AA1FDEF1DF0D9
:103BB000000180BFE8EF1DF011C30DF012C30EF03D
:103BC0007FC00FF080C010F057EC10F0F2EF1DF046
:103BD00015C30DF016C30EF07FC00FF080C010F0BB
:103BE00057EC10F013C30DF014C30EF00001145085
:103BF0000D2615500E2210EF1EF042C30DF043C3E8
:103C00000EF07FC00FF080C010F057EC10F044C3EE
:103C10000DF045C30EF0000114500D2615500E2274
:103C200054EC1EF00DC046F00EC047F081C00DF000
:103C300082C00EF0F40E0D5E010E0E5AD8900D36B5
:103C40000E360EBE2CEF1EF046C30FF047C310F029
:103C500057EC10F032EF1EF04AC30FF04BC310F0D8
:103C600057EC10F048C30DF049C30EF00D50142668
:103C70000E50152214C00DF015C00EF054EC1EF0BD
:103C80000DC048F00EC049F00001CC6753EF1EF0A4
:103C90000301B1516FEC24F0D8A053EF1EF038C3EC
:103CA00040F039C341F012000201AE5100010D5C39
:103CB0000201AF5100010E58E8AE64EF1EF0AEC233
:103CC0000DF0AFC20EF012000201B05100010D5C08
:103CD0000201B15100010E58E8BE1200B0C20DF051
:103CE000B1C20EF01200000133B482EF1EF035A411
:103CF00082EF1EF03594010E5D6E050E37EC0AF072
:103D0000D8801200D89012000001000E0D6E020E35
:103D10000E6E0001000E136E000E146E010E156E75
:103D2000E86A0A6E10EC0CF0020100510001A56F68
:103D300012000001000E0D6E020E0E6E0001000E4C
:103D4000136E000E146E010E156E040E0A6E44EC16
:103D50000CF01200E846E8060B6E0001000E0D6E36
:103D6000030E0E6E0001000E136E000E146E010E97
:103D7000156E0B501426E86A1522100E0A6E10EC10
:103D80000CF01200E846E8060B6E0001000E0D6E06
:103D9000080E0E6E0001000E136E000E146E010E62
:103DA000156E0B501426E86A1522400E0A6E10ECB0
:103DB0000CF00001000EB56F030EB66F0001000E8F
:103DC000B36F030EB46F0001080EB46F100EB76F1F
:103DD00047EC23F00001000E0D6E080E0E6E000180
:103DE000000E136E000E146E010E156E0B5014268D
:103DF000E86A1522010E0A6E44EC0CF01200E84647
:103E0000E8060B6E0001000E0D6E030E0E6E000133
:103E1000000E136E000E146E010E156E0B5014265C
:103E2000E86A15220A6E10EC0CF00001000E0D6E0F
:103E3000040E0E6E0001000E136E000E146E010EC5
:103E4000156E0B50E82A1426E86A15220A6E10EC4B
:103E50000CF01200E846E8060C6E0001000E0D6E34
:103E6000030E0E6E0001000E136E000E146E010E96
:103E7000156E0C501426E86A1522040E0A6E44ECE6
:103E80000CF00001000E0D6E040E0E6E0001000E0F
:103E9000136E000E146E010E156E0C50E82A1426D7
:103EA000E86A1522040E0A6E44EC0CF012000001C0
:103EB000000EB56F030EB66F0001000EB36F060E55
:103EC000B46F000EB76F47EC23F00001000EB56F22
:103ED000040EB66F0001000EB36F070EB46F000E34
:103EE000B76F47EC23F0120002010051E846E806E4
:103EF0000A6E0001000E0D6E030E0E6E0001000E24
:103F0000136E000E146E010E156E0A501426E86A28
:103F10001522010E0A6E44EC0CF0120073C08DF0F5
:103F200074C08EF075C08FF076C090F077C091F0BD
:103F300078C092F079C093F07AC094F07BC095F08D
:103F40007CC096F07DC097F07EC098F07FC099F05D
:103F500080C09AF081C09BF082C09CF012008EEC71
:103F60001FF00301B2516FEC24F0D8B0CAEF1FF07C
:103F7000030EE26E5C0EE16E67EC22F0610EE16E04
:103F800067EC22F0660EE16E67EC22F06B0EE16EDC
:103F900067EC22F08EEC1FF00301B3516FEC24F0BC
:103FA000D8B0EBEF1FF0030EE26E700EE16E67EC1F
:103FB00022F08EEC1FF0750EE16E67EC22F08EECB5
:103FC0001FF07A0EE16E67EC22F08EEC1FF07F0E90
:103FD000E16E67EC22F08EEC1FF00301B4516FEC40
:103FE00024F0D8B006EF20F0030EE26E840EE16EEE
:103FF00067EC22F0890EE16E67EC22F08E0EE16E26
:1040000067EC22F0930EE16E67EC22F012008DC097
:104010000DF08EC00EF010C40FF000010EBE11C4E2
:104020000FF0106A0FBE106857EC10F00001640E1C
:10403000176E000E186E5BEC11F0000113C0E8FF64
:10404000912714C0E8FF922391C00DF092C00EF0AA
:1040500012C40FF000010EBE13C40FF0106A0FBEA1
:10406000106857EC10F00001640E176E000E186E09
:104070005BEC11F0000113C0E8FF8D2714C0E8FFCE
:104080008E2391C00DF092C00EF014C40FF0000109
:104090000EBE15C40FF0106A0FBE106857EC10F07A
:1040A0000001640E176E000E186E5BEC11F000013B
:1040B00013C0E8FF8F2714C0E8FF902393C00DF0D2
:1040C00094C00EF016C40FF000010EBE106A0FBEB1
:1040D000106857EC10F00001640E176E000E186E99
:1040E0005BEC11F0000113C0E8FF8F2714C0E8FF5C
:1040F00090238DC073F08EC074F08FC075F090C0A7
:1041000076F091C077F092C078F093C079F094C0C7
:104110007AF0040117A19BEF20F08FC07DF090C0D2
:104120007EF0040118A19BEF20F000017D1F7E1F8F
:104130007D2BD8B07E2B030198A1B8EF20F08FC063
:104140000DF090C00EF091C00FF092C010F0000181
:104150000DC075F00EC076F00DC077F00EC078F08F
:104160000F507727105078230F50755F1050765BF3
:10417000030199A1D5EF20F08FC00DF090C00EF093
:104180008DC00FF08EC010F000010DC075F00EC094
:1041900076F00DC073F00EC074F00F5073271050FE
:1041A00074230F50755F1050765B03019AA18FEF57
:1041B00021F08DC00DF08EC00EF00DC073F00EC05A
:1041C00074F00DC07FF00EC080F00001640E176E19
:1041D000000E186E03019C51E812D8B43BEF21F099
:1041E000E8BE18EF21F0640800010F6E106A74BF7A
:1041F00006EF21F073C00DF074C00EF057EC10F014
:104200005BEC11F013C073F014C074F0000180AFC8
:104210003BEF21F07FC00DF080C00EF057EC10F0A6
:104220005BEC11F013C07FF014C080F03BEF21F085
:10423000640F00010F6E106A74AF2BEF21F073C092
:104240000DF074C00EF057EC10F05BEC11F013C0E1
:1042500073F014C074F0000180BF3BEF21F07FC009
:104260000DF080C00EF057EC10F05BEC11F013C0B5
:104270007FF014C080F003019BA145EF21F0000105
:104280007F1F801F7F2BD8B0802B0001640E176E1C
:10429000000E186E03019D51E812D8B48FEF21F083
:1042A0000301C651E812D8B468EF21F00301C551EB
:1042B0006FEC24F0D8B08FEF21F00001E80E0D6E06
:1042C000030E0E6E93510D5E94510E5A71EF21F054
:1042D0000001E80E0D6E030E0E6E99510D5E9A519F
:1042E0000E5A9DC30FF09EC310F0106AE8BE101E58
:1042F00057EC10F05BEC11F013507327145074233B
:1043000003019BB18AEF21F00001131E141E132A32
:10431000D8B0142A000113507F27145080231200B4
:104320000301A4A112008EEC1FF007EC20F0120094
:104330000301A4B1A0EF21F08EEC1FF007EC20F0F8
:1043400003019EA1BBEF21F00301C2516FEC24F0E9
:10435000D8A0BBEF21F003019F5100010D6E0E6A42
:1043600000010A0E0F6E000E106E57EC10F013C015
:1043700079F014C07AF00301A0A1E8EF21F0030165
:10438000C3516FEC24F0D8A0CAEF21F00301A15172
:10439000D3EF21F00301C4516FEC24F0D8A0E8EF73
:1043A00021F00301A25100010D6E0E6A00010A0EF8
:1043B0000F6E000E106E57EC10F01350795D145014
:1043C0007A59E8AEE8EF21F013C079F014C07AF022
:1043D00012000BC0E8FFF00BD8B412000DC069F05A
:1043E0000EC06AF00EAEFAEF21F00D1E0E1E0D2A61
:1043F000D8B00E2A0DC013F00EC014F0640E176E64
:104400008AEC10F000011C6A090E136012EF22F012
:104410000BC0E8FFE83AE8060F0BE8B62FEF22F0F2
:1044200024EF22F0136E0DC01BF00EC01CF0840EA2
:1044300000011B5E030E1C5A0BC0E8FFE83AE806B9
:104440000F0BE8B62FEF22F00B0DF350460F13249D
:10445000E8CFD9FF020EE8CFDAFF39EF22F0E89675
:104460000B0DF350DA0F1324E8CFD9FF030EE8CF7A
:10447000DAFFDECF0AF0DFCF0BF000010BC00DF04A
:104480000AC0E8FF0D5E0E6A0DBE0E681BC00FF07D
:104490001CC010F057EC10F00A0E176E8AEC10F0EA
:1044A0000AC0E8FF0A0DF3CFE8FF1326F4CFE8FFB8
:1044B000142213C00DF014C00EF000016AAF1200F8
:1044C00000010D1E0E1E0D2AD8B00E2A1200E65055
:1044D000E8CF0BF0E812D8B4120080EC02F0E9EC5F
:1044E00021F00DC011F00EC012F0E6CF0AF0E6CFB9
:1044F000E8FF0001E8CF0DF00E6A0DBE0E1E0001B0
:104500000A0E0F6E000E106E57EC10F011C00DF079
:1045100012C00EF013500D5E14500E5A0EBEC6EFB0
:1045200022F0E6CFE8FF00010AACAFEF22F0E8CFBF
:1045300013F0E9CF14F00DC011F00EC012F01350BB
:1045400080EC02F00DC013F00EC014F00A0E176ECE
:104550008AEC10F011C00DF012C00EF013500F6E67
:10456000106A0FBE101E57EC10F00001640E176E9B
:10457000000E186E196A1A6A5BEC11F013C00DF088
:1045800014C00EF00A5000EC03F01200E6CFE8FF72
:10459000E6CFE8FF00010AAAE4EF22F0E8CF13F02B
:1045A0000DC011F00EC012F0135080EC02F00DC0DF
:1045B00013F00EC014F00A0E176E8AEC10F011C042
:1045C0000DF012C00EF013500F6E106A0FBE101EC9
:1045D00057EC10F00001640E176E000E186E196A89
:1045E0001A6A5BEC11F013C00DF014C00EF00A5003
:1045F00000EC03F012000001BD0EB56F030EB66FA4
:104600000001120EB36F010EB46F050EB76F47ECC9
:1046100023F0D90EE8CFD9FF060EE8CFDAFF060E59
:10462000E8CF0CF0DDCFE8FFE812D8B41FEF23F09D
:10463000DFCFE8FF6FEC24F0D8B02BEF23F0DDCF15
:10464000E8FF0C2E12EF23F0A5C0E8FF0201006383
:1046500034EF23F01200DECFE8FFDECFE8FF0201E7
:10466000006334EF23F01200E8CF00F2FFEC1EF0FD
:104670000001120EB56F010EB66F0001BD0EB36FD3
:10468000030EB46F050EB76F47EC23F01200000164
:10469000B551E16EB651E26E0001B351D96EB4511D
:1046A000DA6EE6CFE8FFE8CFDEFF0001B72F51EF6B
:1046B00023F012000001BF6B0301AE516FEC24F038
:1046C0000001D8B0BF810301AF516FEC24F00001AD
:1046D000D8B0BF830301B0516FEC24F00001D8B013
:1046E000BF850301B1516FEC24F00001D8B0BF8742
:1046F0000301B6516FEC24F00001D8B0BF8903016B
:10470000BB516FEC24F00001D8B0BF8B0301BC514A
:104710006FEC24F00001D8B0BF8D1200C00E0FEC7A
:104720000DF00301AE516FEC24F00001E86AE8805F
:10473000BF15D8A0AAEF23F0D8A4BBEF23F0BF7118
:10474000000EF86E650EF76E020EF66E75EC0DF04B
:104750006CEF24F0D8B0BBEF23F0D8B4BBEF23F05C
:10476000BF71000EF86E640EF76EF00EF66E75EC0B
:104770000DF06CEF24F00301AF516FEC24F0000159
:10478000E86AE882BF15D8A0D4EF23F0D8A4E5EFFB
:1047900023F0BF73000EF86E650EF76E260EF66EF0
:1047A00075EC0DF06CEF24F0D8B0E5EF23F0D8B441
:1047B000E5EF23F0BF73000EF86E650EF76E140E72
:1047C000F66E75EC0DF06CEF24F00301B0516FEC58
:1047D00024F00001E86AE884BF15D8A0FEEF23F0BA
:1047E000D8A40FEF24F0BF75000EF86E650EF76EBB
:1047F0004A0EF66E75EC0DF06CEF24F0D8B00FEFAA
:1048000024F0D8B40FEF24F0BF75000EF86E650EDB
:10481000F76E380EF66E75EC0DF06CEF24F00301B8
:10482000B1516FEC24F00001D8A025EF24F0BFB700
:1048300026EF24F0BF77000EF86E650EF76E920E2D
:10484000F66E75EC0DF06CEF24F0BF970301B651D6
:104850006FEC24F00001D8A03CEF24F0BFB93DEF8D
:1048600024F0BF79000EF86E650EF76E800EF66EBE
:1048700075EC0DF06CEF24F0BF990301BB516FECA8
:1048800024F00001D8A053EF24F0BFBB54EF24F074
:10489000BF7B000EF86E650EF76E5C0EF66E75EC63
:1048A0000DF06CEF24F0BF9B0301BC516FEC24F0C2
:1048B0000001D8A06AEF24F0BFBD6BEF24F0BF7DEC
:1048C000000EF86E650EF76E6E0EF66E75EC0DF05E
:1048D0006CEF24F0BF9D1200500EA36F1200E8AAE7
:1048E0009BEF24F0E8A89BEF24F00A6E070BC90F9A
:1048F000E16E030EE26EE65000010D6E0E6AE8BE38
:104900000E6800010A0E0F6E000E106E57EC10F0CC
:104910000A50070BE846340FE16E010EE252E650F2
:10492000E6CF0BF00001135E0B501458E8360ABEB8
:104930001200D8701200D890E8BA1200D880E8B8F7
:10494000120000011F6E206AE8BC2080070BE82AD5
:10495000D8802036E82EA9EF24F030501FB633500F
:104960002014D8802062D8901FBED8701200040E88
:10497000D56E1200D59E1200D89087B21200D88052
:10498000D5BE1200C3C00DF0C4C00EF000013C0E35
:104990000F6E000E106E68EC10F013C00DF014C016
:1049A0000EF00001240E0F6EF40E106E68EC10F085
:1049B000C1C017F0C2C018F00001000E196E000E41
:1049C0001A6E3EEC13F0A5C317F0A6C318F0000151
:1049D000186A5BEC11F0C00E0FEC0DF0000EF86ED3
:1049E000640EF76E600EF66E75EC0DF0CB0E0FECEC
:1049F0000DF0DBEC0DF0A5C313F0A6C314F0146AA0
:104A0000C00E0FEC0DF0D7EC0DF00001000EC36FDF
:104A1000000EC46FD88012000001020E3662120030
:104A2000000133A01200FC6A0AEF05F025EC25F026
:104A3000D8A01200FC6A99EC1EF000C2E8FF2AEC34
:104A40001FF057EC1FF00AEF05F0000130B62FEF12
:104A500025F032A62FEF25F03296D8801200D8909C
:104A600012000001650E0E6EB60E0D6E70EC25F094
:104A700054EC0DF00001115080EC01F012001EC149
:104A80000DF01FC10EF054EC0DF012000001EF51BB
:104A9000D8B41200EDEC17F00001000E736F000E99
:104AA000746F0001000E756F000E766FA3EC19F0A5
:104AB00036EC19F070EC1BF002EC1CF001EC1AF073
:104AC00090EC21F0AFEC1FF098EC21F0E7EC1AF03D
:104AD000E3EC1CF04EEC0EF012000001EF69120046
:104AE0000CEC25F00001CD6BDB6BEA6BEB6BC00EC1
:104AF0000FEC0DF00DC0F6FF0EC0F7FFF86A0DC009
:104B00000FF00EC010F075EC0DF0FA0E9DEC0BF0EE
:104B100072EC29F0D8A493EF25F0110E0D26D8B031
:104B20000E2A9AEF25F0D8A0A7EF25F0130E0D2638
:104B3000D8B00E2A0DC0F6FF0EC0F7FFF86A0900C4
:104B4000F5CF0DF00900F5CF0EF077EF25F016EC5C
:104B500025F073EC1EF0D8A077EF25F0150E0D268A
:104B6000D8B00E2A0DC0F6FF0EC0F7FFF86A090094
:104B7000F5CF11F00900F5CF12F00FC00DF010C005
:104B80000EF00900F5CF0FF00900F5CF10F0090085
:104B9000F5CFCEF00900F5CFCFF00001B96BBA6BBD
:104BA000BB697F0EE8CFBCF012ACE3EF25F0090043
:104BB000F5CFB9F00900F5CFBAF00900F5CFBBF099
:104BC0000900F5CFBCF012A4ECEF25F00900F5CFF9
:104BD000EAF00900F5CFEBF012A2F5EF25F009009D
:104BE000F5CFECF00900F5CFEDF012AEFAEF25F0BD
:104BF00054EC0DF012A6FFEF25F06AEC0DF012A2B6
:104C000012000001E86AE8CFFBFFEDC0E8FFE8CF43
:104C1000FAFFECC0E8FFF96EE8CF0AF00FC01BF016
:104C200010C01CF00FC0F6FF10C0F7FFF86A150E99
:104C3000F626D8B0F72A0900F5CFE8FF0A6222EF7E
:104C400026F012000FC0F6FF10C0F7FF110EF62677
:104C5000D8B0F72A0900F5CF0FF00900F5CF10F012
:104C60000FC0E8FF1B6212EF26F010C0E8FF1C62C5
:104C700012EF26F01200000110500F10D8B41200ED
:104C8000E86AFB6E1050E8CFFAFF0F50F96E000192
:104C90000F50E16E1050E26E0001000E116265EFE0
:104CA00026F00FC0F6FF10C0F7FFF86A160EF626C2
:104CB000D8B0F72ACEC0E1FFCFC0E2FFE7CFE8FFD0
:104CC0000CEC26F0DFEC28F01200010E11626CEF04
:104CD00026F00EEC28F01200020E116296EF26F07C
:104CE000000112A077EF26F0CE510001B86FE6CF99
:104CF0000AF0E5CF0BF000010AC011F00BC012F072
:104D0000129E129C64EC28F000010FC0E1FF10C05D
:104D1000E2FF11C00AF012C00BF00AC0E6FFE7CFB5
:104D2000E8FFC00B0B120BC0E5FF1200030E11626F
:104D3000ABEF26F0E7CFE8FFE83667EC27F0000E90
:104D4000D8B0E81E0A6E00010FC0E1FF10C0E2FFFC
:104D50000AC0E7FF1200040E1162BCEF26F0E7CF95
:104D6000E8FF26EC29F00A6E00010FC0E1FF10C039
:104D7000E2FF0AC0E7FF1200050E1162CEEF26F037
:104D8000E7CFE8FFBCEC27F0E8CF0AF000010FC046
:104D9000E1FF10C0E2FF0AC0E7FF1200060E116239
:104DA000E4EF26F0E7CF0AF00FC0CEF010C0CFF04E
:104DB00000016A0E0F6E790E106E0AC0E8FF0CEC4F
:104DC00026F0DFEC28F01200070E1162EBEF26F060
:104DD0003BEC26F01200080E1162FCEF26F0E7CF44
:104DE000E8FFB6EC27F0E8CF0AF000010FC0E1FFC2
:104DF00010C0E2FF0AC0E7FF0A0E11621DEF27F0A4
:104E0000E7CFE8FF0001CE15D890D8B4D88067EC82
:104E100027F00001CEC00AF000010FC0E1FF10C072
:104E2000E2FFD8B018EF27F00AC0E8FFE71212003F
:104E30000AC0E8FFE81EE716120012000B6AD8B09D
:104E40000B1EC00E0FEC0DF0000EF86E640EF76E28
:104E5000060EF66E75EC0DF00BA043EF27F0C80EB2
:104E60000FEC0DF0280E00EC0DF0CC0E0FEC0DF059
:104E7000290E00EC0DF0CF0E0FEC0DF0200E00EC23
:104E80000DF055EF27F0C80E0FEC0DF0200E00ECE2
:104E90000DF0CC0E0FEC0DF0280E00EC0DF0CF0E47
:104EA0000FEC0DF0290E00EC0DF072EC29F0D8B4E7
:104EB0000B6AFF0ED8B00B6E16EC25F073EC1EF0EB
:104EC000D8A02CEF27F0D8900BB0D88012000B6A36
:104ED000D8B00B1EC80E0FEC0DF0000EF86E640E6D
:104EE000F76E440EF66E75EC0DF00BA08CEF27F00C
:104EF000C80E0FEC0DF0280E00EC0DF0CC0E0FECF0
:104F00000DF0290E00EC0DF0CF0E0FEC0DF0200E81
:104F100000EC0DF09EEF27F0C80E0FEC0DF0200E08
:104F200000EC0DF0CC0E0FEC0DF0280E00EC0DF0A7
:104F3000CF0E0FEC0DF0290E00EC0DF072EC29F005
:104F4000D8B40B6AFF0ED8B00B6E16EC25F073ECDC
:104F50001EF0D8A075EF27F0D8900BB0D8801200C3
:104F60000001BB65BB51B961B95112000001E8698C
:104F700000019D6FC0EF27F000019D6F0001E86BFD
:104F8000C80E9DEC0BF09DC0E8FF0001136E146A83
:104F9000156A166A05EC0EF00001E867DEEF27F0EF
:104FA000CD0E0FEC0DF0275000EC0DF0285000EC6A
:104FB0000DF0295000EC0DF0EDEF27F0CC0E0FECCA
:104FC0000DF0275000EC0DF0285000EC0DF02E0EE7
:104FD00000EC0DF0295000EC0DF098EC29F00001E8
:104FE000D8A4F9EF27F09D2BBB519D619D6F04EF75
:104FF00028F0D8A004EF28F09D51B96104EF28F003
:105000009D07B9519D659D6F16EC25F073EC1EF060
:10501000D8A0C0EF27F000019D51120046EC25F00A
:10502000FA0E9DEC0BF0E7CFE8FFE7BEE81EE7BE07
:10503000E82A0001136E146A156A166A05EC0EF070
:10504000CB0E0FEC0DF0200EE7BE2D0E00EC0DF098
:10505000275000EC0DF0285000EC0DF0295000EC2A
:105060000DF0250E00EC0DF098EC29F00001D8A40D
:105070003DEF28F0E72A41EF28F0D8A041EF28F0D3
:10508000E70616EC25F073EC1EF0D8A00EEF28F022
:105090000001EF6B120000011150BB5D1250BC59B2
:1050A000D8B058EF28F0BB51116EBC51126E1200EF
:1050B000B951115CBA511258D8B063EF28F0B95108
:1050C000116EBA51126E12004BEC28F00001BE6B4B
:1050D0000001B851E812D8B476EF28F0B851E16E6B
:1050E000000EE26E11C0E6FF12C0E7FF320E9DEC2B
:1050F0000BF011C013F012C014F0D8901432133218
:10510000156A166A05EC0EF0C90E0FEC0DF026506C
:1051100000EC0DF02E0E00EC0DF0275000EC0DF021
:10512000285000EC0DF0295000EC0DF06D0E00EC55
:105130000DF0530E00EC0DF098EC29F00001D8A40E
:10514000B1EF28F0112AD8B4122A112AD8B4122AA1
:10515000BC51126264EF28F0BB511160116E64EF14
:1051600028F0D8A0C3EF28F01106D8A01206110627
:10517000D8A01206BA51126264EF28F0B951116436
:10518000116E64EF28F0000133A2BE6933BCCEEF8C
:1051900028F00001A00E116E0F0E126E000133BE3A
:1051A000D7EF28F00001D00E116E070E126E16EC2C
:1051B00025F073EC1EF0D8A068EF28F01200C00EA6
:1051C0000FEC0DF00FC0F6FF10C0F7FF75EC0DF0FF
:1051D000FA0E9DEC0BF098EC29F0D8A4F6EF28F02D
:1051E000110E0F26D8B0102AFDEF28F0D8A00AEF34
:1051F00029F0130E0F26D8B0102A0FC0F6FF10C0EA
:10520000F7FFF86A0900F5CF0FF00900F5CF10F0AD
:10521000DFEF28F016EC25F073EC1EF0D8A0DFEFDE
:1052200028F0150E0F26D8B0102A0FC0F6FF10C0B8
:10523000F7FFF86A0900F5CF0AF00900F550CEC073
:10524000E1FFCFC0E2FF0AC0E7FF12000F0BE8B694
:10525000080B0C0DF3CF13F0F4CF14F000019E0EE9
:1052600013266F0E1422CC0E0FEC0DF013C0F6FFB8
:1052700014C0F7FF75EC0DF0FA0E9DEC0BF098ECF6
:1052800029F0D8A44AEF29F0050E1326D8B0142A25
:1052900051EF29F0D8A05EEF29F0070E1326D8B001
:1052A000142A13C0F6FF14C0F7FFF86A0900F5CFFF
:1052B00013F00900F5CF14F033EF29F016EC25F0C8
:1052C00073EC1EF0D8A033EF29F0090E1326D8B0E6
:1052D000142A13C0F6FF14C0F7FFF86A0900F5CFCF
:1052E000E8FF1200040E93EC08F0040E93EC08F0B3
:1052F000C5C0E8FFC35EC6C0E8FFC45AC4BE8BEF9A
:1053000029F0640EC35E000EC45AC4BE95EF29F0A6
:10531000D884D8901200640EC326000EC422C4AEF6
:1053200095EF29F0D894D8801200D894D890120024
:10533000050E93EC08F0050E93EC08F0C7C0E8FFEB
:10534000C35EC8C0E8FFC45AC4BEB1EF29F0640E02
:10535000C35E000EC45AC4BEBBEF29F0D884D890F7
:105360001200640EC326000EC422C4AEBBEF29F0A7
:10537000D894D8801200D894D8901200B8EF2AF0B0
:10538000800E0FEC0DF0000EF86E650EF76ECE0E6F
:10539000F66E75EC0DF005EF2BF00101E60E1E6FB9
:1053A000650E1F6F0101D20E206F670E216F48EC52
:1053B0002AF099EC1EF000C2E8FF2AEC1FF057EC2F
:1053C0001FF012000101FE0E1E6F650E1F6F01011E
:1053D000C40E206F680E216F48EC2AF0D9EF29F037
:1053E0000101160E1E6F660E1F6F0101AE0E206FBB
:1053F0006A0E216F48EC2AF0D9EF29F001012E0E38
:105400001E6F660E1F6F01010A0E206F700E216F56
:1054100048EC2AF0D9EF29F00101460E1E6F660E06
:105420001F6F0101D80E206F760E216F48EC2AF015
:10543000D9EF29F00001DD6B01015E0E1E6F660ED3
:105440001F6F0101E20E206F7C0E216F48EC2AF0E5
:10545000D9EF29F00101760E1E6F660E1F6F010154
:105460002A0E206F810E216F48EC2AF0D9EF29F027
:1054700001018E0E1E6F660E1F6F0101A40E206FBC
:10548000840E216F48EC2AF0D9EF29F036EF31F085
:105490003FEC25F020C10DF021C10EF070EC25F09D
:1054A0000DC020F10EC021F1EAC026F1EBC027F1BA
:1054B00000011150090AD8A4AAEF2AF00FC00DF07C
:1054C00010C00EF070EC25F00DC022F10EC023F1DB
:1054D000EAC028F1EBC029F100011150090AD8A453
:1054E00092EF2AF00FC00DF010C00EF070EC25F016
:1054F0000DC024F10EC025F1EAC02AF1EBC02BF15A
:1055000047EC26F00001CDB198EF2AF02AC10FF048
:105510002BC110F03BEC26F024C10DF025C10EF09C
:1055200076EF2AF047EC26F00001CDB1AFEF2AF07C
:1055300028C10FF029C110F03BEC26F020C10DF07E
:1055400021C10EF054EC0DF022C10DF023C10EF07C
:1055500062EF2AF047EC26F00001CDB1120026C11F
:105560000FF027C110F03BEC26F048EF2AF01200B4
:1055700000C2E8FFAAEC1EF0800E0FEC0DF0000E4A
:10558000F86E630EF76ED00EF66E75EC0DF08D0EA4
:105590000FEC0DF0020100510001136E146A156A40
:1055A000166AD3EC0DF0CDEC05F0FA0E9DEC0BF085
:1055B00098EC29F0D8A4E7EF2AF0610E0201002B45
:1055C0000063B8EF2AF0010E006FB8EF2AF0D8A000
:1055D000F5EF2AF002010007000E0063B8EF2AF091
:1055E000600E0201006FB8EF2AF073EC1EF0D8A035
:1055F000D8EF2AF000C2E8FFFFEC1EF000C2E8FF7F
:10560000E8CFA5F099EC1EF01200C00E0FEC0DF0E3
:10561000CDEC05F0000EE16E030EE26E960E9DECF1
:105620000BF0C00EE1240FEC0DF0E75000EC0DF094
:10563000C00EE1240FEC0DF00E0E0FEC0DF072EC2D
:1056400029F0D8A42DEF2BF0E12A0F0EE1640EEF24
:105650002BF0000EE16E0EEF2BF0D8A039EF2BF0FF
:10566000E106FF0EE1620EEF2BF00F0EE16E0EEF82
:105670002BF098EC29F0D8A444EF2BF0E72A7A0E0F
:10568000E760E76E0EEF2BF0D8A04DEF2BF0E706AA
:10569000200EE764E76E0EEF2BF073EC1EF0D8A03F
:1056A0001FEF2BF00C0E0FEC0DF000C2E8FF2AEC00
:1056B0001FF012000DC02CF10EC02DF10FC02EF105
:1056C00010C02FF1D0C00DF0D1C00EF00001E80ED7
:1056D0000F6E030E106E57EC10F00001000E176EE7
:1056E000010E186E5BEC11F013C0D0F014C0D1F0B5
:1056F0000001D251D027D351D123D4C00DF0D5C051
:105700000EF00001E80E0F6E030E106E57EC10F055
:105710000001000E176E010E186E5BEC11F0D2C086
:10572000D4F0D3C0D5F01350D45F1450D55B2CC146
:105730000DF02DC10EF02EC10FF02FC110F0120090
:105740000DC02CF10EC02DF10FC02EF110C02FF1A5
:10575000D0C00DF0D1C00EF0D2510D5ED3510E5A13
:105760000001000E0F6E010E106E57EC10F00001DC
:10577000E80E176E030E186E5BEC11F013C0D0F03C
:1057800014C0D1F0D2C00DF0D3C00EF0D4510D5ED4
:10579000D5510E5A0001000E0F6E010E106E57EC1F
:1057A00010F00001E80E176E030E186E5BEC11F09E
:1057B00013C0D4F014C0D5F02CC10DF02DC10EF0E3
:1057C0002EC10FF02FC110F012000DC02CF10EC031
:1057D0002DF10FC02EF110C02FF10001BEA11DEF61
:1057E0002CF0000E00010F18D8B408EF2CF0D2C036
:1057F00013F0D3C014F0D89013361436D051135E82
:10580000D151145A13C0D4F014C0D5F01DEF2CF0B0
:10581000000E00010F18D8B41DEF2CF0D2C013F009
:10582000D3C014F0D89013361436D451135ED5512A
:10583000145A13C0D0F014C0D1F02CC10DF02DC1FA
:105840000EF02EC10FF02FC110F012003C0E00011F
:10585000B86F0001110EB56F030EB66F0001D00EC8
:10586000B36F000EB46F0B0EB76F47EC23F0DB6B1A
:105870005AEC2BF012003A0E0001B86F00011C0E1A
:10588000B56F030EB66F2EEF2CF03E0E0001B86F11
:105890000001270EB56F030EB66F2EEF2CF000013E
:1058A000110EB36F030EB46FE5EC2BF0DBA1D86BD8
:1058B000A0EC2BF00001D00EB56F000EB66F0B0EF2
:1058C000B76F47EC23F00001B86B120000011C0E0B
:1058D000B36F030EB46F54EF2CF00001270EB36FBB
:1058E000030EB46F54EF2CF00DC02CF10EC02DF14F
:1058F0000FC02EF110C02FF1030132C30DF033C3DE
:105900000EF00001E80E0F6E030E106E57EC10F053
:105910000001000E176E010E186E5BEC11F013C043
:1059200032F314C033F3030134513227355133239A
:105930002CC10DF02DC10EF02EC10FF02FC110F0B3
:1059400012000DC02CF10EC02DF10FC02EF110C0B1
:105950002FF132C30DF033C30EF0030134510001B7
:105960000D5E0301355100010E5A0001000E0F6E4D
:10597000010E106E57EC10F00001E80E176E030ECA
:10598000186E5BEC11F013C032F314C033F32CC16A
:105990000DF02DC10EF02EC10FF02FC110F000013F
:1059A000B86B1200420E0001B86F00013A0EB56FDD
:1059B000030EB66F0001D00EB36F000EB46F040E6D
:1059C000B76F47EC23F05AEC2BF01200440E0001A5
:1059D000B86F00013E0EB56F030EB66FDAEF2CF014
:1059E000460E0001B86F0001420EB56F030EB66F90
:1059F000DAEF2CF000013A0EB36F030EB46FA0EC97
:105A00002BF00001D00EB56F000EB66F040EB76F0D
:105A100047EC23F00001B86B120000013E0EB36F9B
:105A2000030EB46FFFEF2CF00001420EB36F030EB4
:105A3000B46FFFEF2CF00001460EB56F030EB66F8A
:105A40000001D00EB36F000EB46F060EB76F47ECB7
:105A500023F05AEC2BF01200A0EC2BF00001D00E3A
:105A6000B56F000EB66F0001460EB36F030EB46F34
:105A7000060EB76F47EC23F00001B86B1200AEC200
:105A8000B9F0AFC2BAF0B0C2BBF0B1C2BCF0120004
:105A9000CEC0B5F0CFC0B6F00001DC0EB36F000E83
:105AA000B46F050EB76F47EC23F0CEC0B3F0CFC094
:105AB000B4F00001DC51E83A0F0BE46FE36BDDBF9B
:105AC000E31FE16BDF51DDBDE16FE26BE051DDBB58
:105AD000E26F0F0EE117E217DD17DC17120000016D
:105AE000E451E83AF00BDC13E3BFDD8FE151E8123B
:105AF000D8B47EEF2DF0E151DF6FDD8DE251E81279
:105B0000D8B486EF2DF0E251E06FDD8B0001DC0EA2
:105B1000B56F000EB66F050EB76F47EC23F012009D
:105B200010C4DFF011C4E0F01200DFC010F4E0C0D8
:105B300011F4120012C4DFF013C4E0F01200DFC051
:105B400012F4E0C013F4120014C4DFF015C4E0F046
:105B50001200DFC014F4E0C015F412000001DBAF46
:105B600012000301196B246B2F6B12000001DBAFD5
:105B70001200A7C313F0A8C314F083511326845155
:105B8000142213C0A7F314C0A8F3A9C313F0AAC327
:105B900014F0855113268651142213C0A9F314C0A2
:105BA000AAF3ABC313F0ACC314F08751132688518A
:105BB000142213C0ABF314C0ACF312000001DBAF2E
:105BC00012000301A76BA86BA96BAA6BAB6BAC6B44
:105BD00012000001B96BB92B600E0001BB6F1200FF
:105BE0000001DD51DD67F6EF2DF01200020100C269
:105BF0000AF0006F00010AC0DDF02AEC1FF000017E
:105C0000DDC00AF002010AC000F212000001DBAFA1
:105C1000120003011951196B18C30AF000010D6E2F
:105C20000E6AE8BE0E680D360E360001640E0F6E69
:105C3000000E106E57EC10F00AC017F0186A5BECFB
:105C400011F013500301A727000114500301A823EA
:105C500003012451246B23C30AF000010D6E0E6A68
:105C6000E8BE0E680D360E360001640E0F6E000E93
:105C7000106E57EC10F00AC017F0186A5BEC11F0C8
:105C800013500301A927000114500301AA230301A3
:105C90002F512F6B2EC30AF000010D6E0E6AE8BE65
:105CA0000E680D360E360001640E0F6E000E106E7B
:105CB00057EC10F00AC017F0186A5BEC11F01350A3
:105CC0000301AB27000114500301AC2312000001B3
:105CD000DBAF120097EC31F0120047EC23F012001A
:105CE0000001D00EB36F000EB46FCEC0B5F0CFC0C0
:105CF000B6F00B0EB76F47EC23F00001D00EB56F76
:105D0000000EB66FCEC0B3F0CFC0B4F00B0EB76FBD
:105D100012000201D890A23712000201D890A233DB
:105D200012000001E9AF120001EC10F0120013C2E2
:105D30000FF014C210F0030E0001A06F46EC30F01B
:105D40000FC013F210C014F21200A9C20FF0AAC2C1
:105D500010F00D0E0001A06F46EC30F00FC0A9F25C
:105D600010C0AAF212000001DBAF12000501006BA7
:105D7000016B1200C9EC0BF012000001CE51B36FA1
:105D8000020EB46FCF5100011F6E030E7EEC08F0BF
:105D900014C08BF015C08CF0C00E0FEC0DF0000E8F
:105DA000F86E8A0EF76EBC0EF66E75EC0DF073ECA5
:105DB0001EF0D8A0D7EF2EF000011F507EEC08F0A7
:105DC00014C06DF015C06EF014C06FF015C070F007
:105DD000FA0E9DEC0BF0C00E0FEC0DF0000EF86EFD
:105DE0008A0EF76ECE0EF66E75EC0DF073EC1EF0AB
:105DF000D8A0F6EF2EF000011F507EEC08F014C082
:105E00006BF015C06CF0FA0E9DEC0BF000016B51BD
:105E10006D276C516E236E336D336E9F6FC017F01C
:105E200070C018F00001E80E146E030E156E136AB0
:105E3000166A6B51175E6C51185A18321732189E39
:105E4000196A1A6A5BEC11F013C06BF014C06CF0A5
:105E500000016B0EB56F000EB66F040E0001B76F38
:105E600047EC23F012000001CE51B36F020EB46F65
:105E7000CF5100011F6EC00E0FEC0DF0000EF86E3A
:105E80008A0EF76EBC0EF66E75EC0DF073EC1EF01C
:105E9000D8A046EF2FF000011F507EEC08F014C090
:105EA0006BF015C06CF0FA0E9DEC0BF0C00E0FEC11
:105EB0000DF0000EF86E8A0EF76ECE0EF66E75ECD3
:105EC0000DF073EC1EF0D8A061EF2FF000011F5011
:105ED0007EEC08F014C06DF015C06EF0FA0E9DEC6B
:105EE0000BF00001E80E146E030E156E136A166AAD
:105EF0006BC017F06CC018F0196A1A6A00016D5176
:105F0000175E6E51185A18AE87EF2FF0FF0E196EFC
:105F10001A6E5BEC11F013C06BF014C06CF0000152
:105F20006B0EB56F000EB66F040E0001B76F47EC35
:105F300023F012000001CE51B36F020EB46FCF51A7
:105F400000011F6EC00E0FEC0DF0000EF86E8A0EF1
:105F5000F76EAA0EF66E75EC0DF073EC1EF0D8A07D
:105F6000ADEF2FF000011F507EEC08F0000113365A
:105F70001436153614C06DF015C06EF0FA0E9DEC97
:105F80000BF0C00E0FEC0DF0000EF86E8A0EF76EDF
:105F9000BC0EF66E75EC0DF073EC1EF0D8A0CCEFD5
:105FA0002FF000011F507EEC08F00001133614366C
:105FB000153614C06BF015C06CF0FA0E9DEC0BF0AA
:105FC000C00E0FEC0DF0000EF86E8A0EF76ECE0EBE
:105FD000F66E75EC0DF073EC1EF0D8A0EBEF2FF021
:105FE00000011F507EEC08F0000113361436153600
:105FF00014C06FF015C070F0FA0E9DEC0BF00001AC
:10600000E80E146E030E156E136A166A6BC017F055
:106010006CC018F0196A1A6A00016D51175E6E5152
:10602000185A18AE15EF30F0FF0E196E1A6E5BECB1
:1060300011F013C06BF014C06CF00001E80E146E88
:10604000030E156E136A166A6DC017F06EC018F055
:10605000196A1A6A00016F51175E7051185A18AE0A
:1060600033EF30F0FF0E196E1A6E5BEC11F013C0B7
:106070006FF014C070F000016B0EB56F000EB66FBC
:10608000060E0001B76F47EC23F01200140E9DECD2
:106090000BF00001A05193EC08F0C00E0FEC0DF0D6
:1060A000000EF86E670EF76E660EF66E75EC0DF06C
:1060B000CB0E0FEC0DF069C00DF06AC00EF057EC7E
:1060C00010F01450136E1550146E156A05EC0EF096
:1060D000200E0A6E300E25640AC025F0255000EC13
:1060E0000DF0265000EC0DF02E0E00EC0DF02750B8
:1060F00000EC0DF0285000EC0DF098EC29F0D8A43D
:1061000088EF30F000010F2AD8B4102A46EF30F0A3
:10611000D8A092EF30F000010F06FF0E0F601006BE
:1061200046EF30F073EC1EF0D8A046EF30F01200CE
:106130000201FF0EA563AAEF30F000019D510FECA4
:106140000DF0000EF86E630EF76EF40EF66E75EC41
:106150000DF012000201D1B1C8EF30F0D1A3C8EFA9
:1061600030F000019D510FEC0DF0000EF86E630E43
:10617000F76EE20EF66E75EC0DF000019D51080F02
:106180000FEC0DF00201310EA52500EC0DF0120010
:106190000201D1A1FDEF30F0D1B3FDEF30F00001ED
:1061A0009D510FEC0DF0000EF86E640EF76E4E0E62
:1061B000F66E75EC0DF000019D510E0F0FEC0DF019
:1061C0000201300EA52500EC0DF00201A551D8907A
:1061D000E836500F0001136E146A156A166A05EC52
:1061E0000EF000019D51040F0FEC0DF0285000EC53
:1061F0000DF0295000EC0DF012000201D1A11200A7
:10620000D1A3120000019D510FEC0DF0000EF86EAD
:10621000640EF76EBA0EF66E75EC0DF000019D512E
:106220000D0F0FEC0DF00201A55101010E2500012B
:10623000136E146A156A166AD3EC0DF00201A551AB
:10624000D890E836010F0001136E146A156A166AB9
:1062500005EC0EF000019D51040F0FEC0DF02850DD
:1062600000EC0DF0295000EC0DF012000301FF0EC0
:10627000AD634BEF31F0C00E0FEC0DF0000EF86E79
:10628000630EF76EF40EF66E75EC0DF0FA0E9DECE3
:106290000BF057EF31F00301AD510201A56FC00EB5
:1062A00000019D6F98EC30F0FA0E9DEC0BF098EC2D
:1062B00029F0D8A467EF31F0010110510301AD2B93
:1062C000AD6336EF31F0FF0EAD6F36EF31F0D8A091
:1062D00077EF31F00301AD07FE0EAD6336EF31F01D
:1062E00001011051E8060301AD6F36EF31F073EC98
:1062F0001EF0D8A057EF31F000C2E8FF2AEC1FF0E3
:106300001200000EF86E8A0EF76EE00EF66E000EAA
:106310000A6E020EE26E000EE16E0900F550E66EA6
:106320000A060900F550E66E0A2E8DEF31F0000ED8
:10633000F86E8B0EF76EE00EF66E000E0A6E030E10
:10634000E26E000EE16E0900F550E66E0A060900E5
:10635000F550E66E0A2EA3EF31F0000EF86E8C0EAB
:10636000F76EE00EF66E000E0A6E040EE26E000E80
:10637000E16E0900F550E66E0A060900F550E66E7A
:106380000A2EB9EF31F012002020202020202020FA
:1063900020202020202020200000204D6963726FE3
:1063A0005374617220323030302000002020566556
:1063B0007273696F6E20322E3064202000004144D9
:1063C00043204348205858203D2058585858000032
:1063D000202020416972637261667420232020208E
:1063E0000000202020202035332E58204D487A20D0
:1063F00020200000202020202020204F4646202062
:10640000202020200000204163636570743F2059E4
:106410006573204E6F20000020507265737320203A
:10642000204F7074696F6E200000202020202020F3
:1064300020002020202053747564656E7420202075
:106440002020000020596573204E6F200000203569
:10645000302E5858204D487A2020434858200000BC
:1064600078426C642052504D203D207878787878BE
:106470000000526574726163747320617265205507
:10648000502100002020466F726D617420466C61BF
:106490007368202000002020466F726D6174696E61
:1064A000672E2E2E20200000202020436F70796957
:1064B0006E672E2E2E20202000002037322E5858B6
:1064C000204D487A20434858582000005245432028
:1064D000566F6C74733D2058582E585800005468FD
:1064E000726F74746C65202041646A757374000067
:1064F000202041494C20442F522048494748202021
:106500000000202041494C20442F5220204C4F575E
:10651000202000002020454C4520442F522048498F
:106520004748202000002020454C4520442F522081
:10653000204C4F5720200000202052554420442F4B
:10654000522048494748202000002020525544202E
:10655000442F5220204C4F57202000002020205351
:106560004E4150205249474854202020000020200E
:1065700020534E415020204C4546542020200000FE
:106580002020204155544F20205452494D20202096
:106590000000202020202050524553455420202028
:1065A0002020000020202043414C494252415445C4
:1065B00020202020000053656C6563742020416911
:1065C00072637261667400CE65BE66000000204191
:1065D0006972637261667420206E616D652000E6E9
:1065E00065B66504000020202020202054696D65D8
:1065F00072202020202000FE65CE650800002020AB
:1066000020202020536E61702020202020200016A2
:1066100066E6650C00002020202020536572766F0E
:10662000732020202020002E66FE65100000202010
:106630002020204D6978657273202020202000469C
:1066400066166614000020202020205377697463AA
:10665000682020202020005E662E66180000202082
:1066600020204F7074696F6E7320202020200076E8
:106670006646661C000020536861726564204F7096
:1066800074696F6E7320008E665E662000002020A5
:1066900053797374656D205365747570202000A65E
:1066A00066766624000053656C65637420467265E7
:1066B0007175656E637900BE668E662800002020C5
:1066C000202020204558495420202020202000B69A
:1066D00065A6662C0000456E61626C652020202056
:1066E00020202020202000005265736574203F2068
:1066F000202020202020202000005A65726F2020BA
:106700003F2020202020202020200000436C6561B5
:1067100072203F20202020202020202000004169DE
:1067200072637261667420232020202020200000E4
:10673000546F204146542023202020202020202058
:106740000000426C61646573203D202020202020E1
:106750002020000046786420467273742020202098
:10676000202020200000566F6C74732020202020F1
:1067700020202020202000005769647468202020F9
:10678000202020202020202000004368616E6E65BC
:106790006C73202020202020202000004E656753AD
:1067A000686966743F202020202020200000506F60
:1067B00073203D20202020202020202020200000A9
:1067C0004761696E202020202020202020202020CA
:1067D00000002020202020204D6F646520202020F4
:1067E000202000EE67626800807C68BD03004D6970
:1067F0006E75746573202020202020202020000E3C
:1068000068D2670540BF0300000000FF0000536529
:10681000636F6E6473202020202020202020002E13
:1068200068EE670540BE0300000000FF0000204541
:106830006E61626C6520205377697463682000483C
:10684000680E680680C003005468726F74746C65CB
:1068500020202020202020200062682E680100C116
:1068600003004558495420202020202020202020AB
:10687000202000D26748680300CD0000202020209F
:1068800055502054696D657220202020009468AC1A
:1068900068000000202020446F776E2054696D65E9
:1068A0007220202000AC687C68010000446F776E85
:1068B000202053746F702054696D6572007C689459
:1068C0006802000053522041494C20202020202003
:1068D0002020202000E468946A01404C030000FF5F
:1068E000007E0000535220454C45202020202020CF
:1068F00020202020000469C46801404E030000FFEE
:10690000007E000053522052554420202020202099
:1069100020202020002469E468014050030000FF8B
:10692000007E000053522054485420202020202074
:10693000202020200044690469014052030000FF28
:10694000007E000053522041494C203F202020204F
:1069500020202020005E69246903004D030053526B
:1069600020454C45203F202020202020202000785A
:1069700069446903004F0300535220525544203F9D
:1069800020202020202020200092695E69030051F1
:106990000300535220544854203F20202020202020
:1069A000202000AC6978690300530300534C204158
:1069B000494C2020202020202020202000CC69923B
:1069C00069014054030000FF007E0000534C204545
:1069D0004C452020202020202020202000EC69ACE5
:1069E00069014056030000FF007E0000534C205216
:1069F000554420202020202020202020000C6ACC7C
:106A000069014058030000FF007E0000534C2054F1
:106A1000485420202020202020202020002C6AEC18
:106A20006901405A030000FF007E0000534C2041E2
:106A3000494C203F202020202020202000466A0CA6
:106A40006A0300550300534C20454C45203F20204D
:106A500020202020202000606A2C6A0300570300B9
:106A6000534C20525544203F20202020202020201D
:106A7000007A6A466A0300590300534C2054485474
:106A8000203F202020202020202000946A606A03DC
:106A9000005B03004558495420202020202020205E
:106AA0002020202000C4687A6A0300CD0000202046
:106AB000202041696C65726F6E202020202000CE5E
:106AC0006AC86B0986E26B00009E584C5800202073
:106AD0002020456C657661746F722020202000EEC6
:106AE0006AAE6A0986E26B0000CC58765800202016
:106AF0002020205275646465722020202020000E22
:106B00006BCE6A0986E26B0000DA588A58002020B2
:106B100020205468726F74746C6520202020002E31
:106B20006BEE6A0986D86C00004259E858002020B4
:106B30002020202043483520202020202020004EE7
:106B40006B0E6B0986CA6D0000F459A45900202011
:106B50002020202043483620202020202020006EA6
:106B60006B2E6B0986CA6D00001A5ACC5900202082
:106B70002020202043483720202020202020008E65
:106B80006B4E6B0986CA6D0000285AE05900202020
:106B9000202020204348382020202020202000AE24
:106BA0006B6E6B0986206E0000585A365A00202002
:106BB0002020537562205472696D7320202000C814
:106BC0006B8E6B0980946E0045584954202020201C
:106BD000202020202020202000AE6AAE6B0300CDB4
:106BE000000052542F44574E2020202020202020E7
:106BF000202000006CBE6C0202D00000007E5A0013
:106C000043656E74657220202020202020202020E3
:106C1000001E6CE26B0202D20000007E5A004C544F
:106C20002F55502020202020202020202020003CF4
:106C30006C006C0202D40000007E5A004475616C46
:106C400020526174652020202020202000566C1ED8
:106C50006C0100D600005472696D20202020202095
:106C600020202020202000706C3C6C0100D7000008
:106C70004154205253542020202020202020202026
:106C8000008A6C566C0300DB00004578706F20486A
:106C90004920202020202020202000A46C706C019E
:106CA00000D900004578706F204C4F5720202020DD
:106CB0002020202000BE6C8A6C0100DA00004558BC
:106CC000495420202020202020202020202000E2C5
:106CD0006BA46C0300CD0000486967682020202069
:106CE000202020202020202000F66C686D02033236
:106CF0000340007E5A004C6F772020202020202067
:106D000020202020202000146DD86C020334034082
:106D1000007E5A005472696D2020202020202020FF
:106D200020202020002E6DF66C01003603005472E6
:106D3000696D204D6F646520202020202020004AAE
:106D40006D146D0000826D370300507265736574B9
:106D50002020202020202020202000686D2E6D0281
:106D600003380340007E5A00455849542020202013
:106D7000202020202020202000D86C4A6D0300CD48
:106D800000005472696D204D6F6465204E4F524D66
:106D9000414C009A6DB26D0000005472696D204D37
:106DA0006F6465202020204C4F5700B26D826D012A
:106DB00000005472696D204D6F64652020204849A1
:106DC000474800826D9A6D020000486967682F5538
:106DD0007020202020202020202000E86D066E0258
:106DE00002D00000007E5A004C6F772F44574E208F
:106DF000202020202020202000066ECA6D0202D212
:106E00000000007E5A0045584954202020202020B0
:106E100020202020202000CA6DE86D0300CD000056
:106E20004120202020202020202020202020202041
:106E3000003E6E7A6E0203D00048007E5A00422067
:106E40002020202020202020202020202020005C26
:106E50006E206E0203D20048007E5A00432020209C
:106E6000202020202020202020202020007A6E3E7C
:106E70006E0203D40048007E5A0045584954202031
:106E80002020202020202020202000206E5C6E0367
:106E900000CD000041696C65726F6E2020202020BB
:106EA0002020202000B26E846F010208040000DA66
:106EB0004A00456C657661746F7220202020202086
:106EC000202000D06E946E010209040000DA4A000E
:106ED000527564646572202020202020202020200C
:106EE00000EE6EB26E01020A040000DA4A00546835
:106EF000726F74746C652020202020202020000CEC
:106F00006FD06E01020B040000DA4A0043483520BE
:106F1000202020202020202020202020002A6FEE6A
:106F20006E01020C040000DA4A004348362020209B
:106F30002020202020202020202000486F0C6F01DE
:106F4000020D040000DA4A004348372020202020A8
:106F5000202020202020202000666F2A6F01020EB2
:106F6000040000DA4A004348382020202020202056
:106F700020202020202000846F486F01020F040091
:106F800000DA4A0045786974202020202020202043
:106F90002020202000946E666F0300CD00004E6F0D
:106FA0006E6500AA6FFE6F0000002041494C00B6DC
:106FB0006F9E6F01000020454C4500C26FAA6F0212
:106FC00000002052554400CE6FB66F0300002054DD
:106FD000485400DA6FC26F0400002043483500E6D1
:106FE0006FCE6F0500002043483600F26FDA6F065F
:106FF00000002043483700FE6FE66F070000204383
:107000004838009E6FF26F080000202020204D4974
:1070100058455220314120202020002A70C2720998
:10702000862A735C03DE5A905A00202020204D49A6
:1070300058455220314220202020004A700A700911
:10704000862A736103DE5A905A00202020204D4981
:1070500058455220314320202020006A702A7009B0
:10706000862A736603DE5A905A00202020204D495C
:1070700058455220314420202020008A704A70094F
:10708000862A736B03DE5A905A00202020204D4937
:107090005845522032412020202000AA706A7009F1
:1070A000862A737003DE5A905A00202020204D4912
:1070B0005845522032422020202000CA708A700990
:1070C000862A737503DE5A905A00202020204D49ED
:1070D0005845522032432020202000EA70AA70092F
:1070E000862A737A03DE5A905A00202020204D49C8
:1070F00058455220324420202020000A71CA7009CD
:10710000862A737F03DE5A905A00202020204D49A2
:1071100058455220334120202020002A71EA70096E
:10712000862A738403DE5A905A00202020204D497D
:1071300058455220334220202020004A710A71090C
:10714000862A738903DE5A905A00202020204D4958
:1071500058455220334320202020006A712A7109AB
:10716000862A738E03DE5A905A00202020204D4933
:1071700058455220334420202020008A714A71094A
:10718000862A739303DE5A905A0020202041494CEE
:1071900020746F2052554420202000AA716A710982
:1071A00086DC7293032A5B205B002020205255442A
:1071B00020746F2041494C20202000CA718A710937
:1071C00086DC7293033E5B345B00202020525544E2
:1071D00020746F20454C4520202000EA71AA7109D7
:1071E00086DC729303525B485B0020202054485495
:1071F00020746F20454C45202020000672CA710182
:10720000881604C067002020202020565441494C95
:10721000202020202020002272EA7103889803D6C3
:1072200066002020202020454C45564F4E2020202F
:107230002020003E72067203889903D66600202043
:1072400020204455414C2041494C2020202000580A
:107250007222720980307400202020204455414C55
:1072600020454C45202020200072723E720980CCBF
:1072700074002020202054485420484F4C442020A3
:107280002020008C72587209801A7500202020205E
:1072900049444C45202055502020202000A67272E1
:1072A00072098068750020204D6978657220206F12
:1072B00072646572202000C2728C720388A4035429
:1072C00067004558495420202020202020202020DD
:1072D0002020000A70A6720300CD0000506F7320BA
:1072E0006761696E202020202020202000F6721087
:1072F000730100DF00004E6567206761696E202022
:10730000202020202020001073DC720100E000000B
:1073100045584954202020202020202020202020B3
:1073200000DC72F6720300CD000046726F6D202003
:1073300020202020202020202020004473167404C8
:1073400000DC00005461626C652020202020202099
:10735000202020200060732A730000D075E4000014
:10736000546F20202020202020202020202020209A
:10737000007A7344730400DD00005265706C616331
:10738000652020202020202020200094736073039B
:1073900000E300005A502020202020202020202020
:1073A0002020202000AE737A730100DE0000506FB1
:1073B00073206761696E202020202020202000C8D3
:1073C0007394730100DF0000506F7320496E6420D6
:1073D000202020202020202000E273AE730400E152
:1073E00000004E6567206761696E20202020202004
:1073F000202000FC73C8730100E000004E65672088
:10740000496E64202020202020202020001674E2D5
:10741000730400E200004558495420202020202019
:10742000202020202020002A73FC730300CD0000C0
:10743000456E61626C6520202020202020202020C5
:10744000004A74B27403009A0300526576204348E0
:107450003720202020202020202000647430740356
:10746000009B030044494646202020202020202065
:1074700020202020007E744A7401009C0300466C8A
:107480006170202020202020202020202020009813
:1074900074647401009D030043524F572020202044
:1074A000202020202020202000B2747E740300C6FB
:1074B000030045584954202020202020202020204F
:1074C000202000307498740300CD0000456E616286
:1074D0006C652020202020202020202000E6740041
:1074E000750300170400526576204348362020209B
:1074F000202020202020000075CC740300180400F8
:1075000045584954202020202020202020202020C1
:1075100000CC74E6740300CD0000456E61626C65BA
:10752000202020202020202020200034754E7503AC
:10753000009E0300506F736974696F6E20202020D5
:1075400020202020004E751A7501009F0300455829
:107550004954202020202020202020202020001AF4
:107560007534750300CD0000456E61626C652020A6
:107570002020202020202020008275B6750300A046
:107580000300506F736974696F6E204120202020C2
:107590002020009C7568750100A10300506F73697D
:1075A00074696F6E204220202020202000B6758252
:1075B000750100A2030045584954202020202020B6
:1075C0002020202020200068759C750300CD00003D
:1075D0005461626C65202020202020204E6F6E6553
:1075E00000E875C0760000004169726372616674DC
:1075F000205461626C652031000076D0750900006E
:107600004169726372616674205461626C652032F4
:10761000001876E8750A0000476C6F6162616C20A3
:107620005461626C652020310030760076010000E4
:10763000476C6F6162616C205461626C652020321E
:107640000048761876020000476C6F6162616C201A
:107650005461626C65202033006076307603000050
:10766000476C6F6162616C205461626C65202034EC
:107670000078764876040000476C6F6162616C2088
:107680005461626C652020350090766076050000BC
:10769000476C6F6162616C205461626C65202036BA
:1076A00000A8767876060000476C6F6162616C20F6
:1076B0005461626C6520203700C076907607000028
:1076C000476C6F6162616C205461626C6520203888
:1076D00000D075A876080000202020202041494CC9
:1076E000204452202020202000F276C6780680AE6A
:1076F00003002020202020454C45204452202020FB
:107700002020000C77D8760680AF030020202020B0
:10771000205255442044522020202020002677F279
:10772000760680B00300202020202050524553458B
:107730005420202020200040770C770680B10300E1
:10774000202020204D495845522020312020202043
:10775000005A7726770680B20300202020204D496A
:107760005845522020322020202000747740770690
:1077700080B30300202020204D495845522020335B
:1077800020202020008E775A770680B40300202026
:10779000202020204348352020202020202000A821
:1077A0007774770680B50300202020204155544F80
:1077B000205452494D20202000C2778E770680B693
:1077C0000300202020202043483820412020202072
:1077D000202000DC77A8770680B703002020202037
:1077E00020434838204220202020202000F677C265
:1077F000770680B80300202020202043483820430B
:10780000202020202020001078DC770680B903009B
:1078100020202020534E4150202052202020202084
:10782000002A78F6770680BB030020202020534EE4
:10783000415020204C202020202000447810780641
:1078400080BC0300205468726F74746C65202048FB
:107850006F6C6420005E782A780680C203002020C6
:107860002049646C6520557020203120202000784C
:107870007844780680C3030020202049646C65208A
:1078800055702020322020200092785E780680C437
:10789000030020202020202043524F57202020206A
:1078A000202000AC7878780680C5030020547269E7
:1078B0006767657220506F696E74732000C6789296
:1078C000780980E078004558495420202020202065
:1078D00020202020202000D876AC780300CD0000A6
:1078E00041696C65726F6E205472696720506F73C6
:1078F00000FC7850790188C903AE6700456C657655
:1079000061746F722054726720506F73001879E0B1
:10791000780188CA03AE67005275646465722020DE
:107920005472696720506F73003479FC780188CBFA
:1079300003AE67005468726F74746C65205472678C
:1079400020506F7300507918790188CC03AE67001E
:10795000455849542020202020202020202020206D
:1079600000E07834790300CD000020202020202082
:10797000204F4E20202020202020008279CA7C1019
:107980000000202020202020204F464620202020BC
:107990002020009A796A7920000053574120202046
:1079A00020202020202020204F4E00B27982790014
:1079B0000000535741202020202020202020204F4D
:1079C000464600CA799A7980000053574220202009
:1079D00020202020202020204F4E00E279B2790183
:1079E0000000535742202020202020202020204F1C
:1079F000464600FA79CA7981000053574320202077
:107A000020202020202020204F4E00127AE27902F0
:107A10000000535743202020202020202020204FEA
:107A20004646002A7AFA79820000535744202020E3
:107A30002020202020505245535300427A127A834E
:107A4000000053574420202020202052454C45411F
:107A50005345005A7A2A7A030000535745202020C4
:107A600020202020202020204F4E00727A427A04CD
:107A70000000535745202020202020202020204F88
:107A80004646008A7A5A7A840000535746202020BE
:107A900020202020202020204F4E00A27A727A053C
:107AA0000000535746202020202020202020204F57
:107AB000464600BA7A8A7A8500005357472020202C
:107AC00020202020202020204F4E00D27AA27A06AB
:107AD0000000535747202020202020202020204F26
:107AE000464600EA7ABA7A8600005357482020209A
:107AF00020202020202020204F4E00027BD27A0719
:107B00000000535748202020202020202020204FF4
:107B10004646001A7BEA7A87000053574920202006
:107B20002020202020505245535300327B027B8975
:107B3000000053574920202020202052454C454129
:107B40005345004A7B1A7B09000053574A202020E6
:107B50002020202020202020204100627B327B8BAF
:107B6000000053574A2020202020202020202020C1
:107B70002042007A7B4A7B4B000053574A2020204A
:107B80002020202020202020204300927B627B8C1C
:107B9000000053574B202020202020202020202090
:107BA0004F4E00AA7B7A7B0D000053574B202020BC
:107BB000202020202020204F464600C27B927B8D33
:107BC000000053574C2020202020202020505245D8
:107BD000535300DA7BAA7B8E000053574C202020A1
:107BE00020202052454C4541534500F27BC27B0E7C
:107BF000000053574D2020202020202020505245A7
:107C00005353000A7CDA7B8F000053574D2020200D
:107C100020202052454C4541534500227CF27B0FE9
:107C2000000041696C65726F6E20202020202020AA
:107C30004F4E003A7C0A7C30000041696C65726FDF
:107C40006E2020202020204F464600527C227CB00F
:107C50000000456C657661746F7220202020202022
:107C60004F4E006A7C3A7C310000456C6576617449
:107C70006F7220202020204F464600827C527CB12B
:107C8000000052756464657220202020202020208E
:107C90004F4E009A7C6A7C320000527564646572B3
:107CA000202020202020204F464600B27C827CB23B
:107CB00000005468726F74746C65202020202020AE
:107CC0004F4E00CA7C9A7C3300005468726F747403
:107CD0006C6520202020204F4646006A79B27CB394
:107CE00000002020204175746F20205472696D209F
:107CF000202000FC7C067E0980967F00526573651B
:107D000074204175746F205472696D73001A7DE29E
:107D10007C038CDB00E8665C5B00202020547269E9
:107D20006D20205A65726F20202000387DFC7C0376
:107D30008CDB00FA666C5B00436C656172205472E8
:107D4000696D205A65726F7300567D1A7D038CDB56
:107D5000000C67BC5B0020416C74202020416972DC
:107D600063726166742000707D387D0980207E001A
:107D700020436F70792020416972637261667420BC
:107D800000907D567D058EDD003067E05BD25B00A4
:107D900020205365742044656661756C74732020DF
:107DA00000AE7D707D038CDB00E866CE5C004E7516
:107DB0006D202070726F7020626C6164657300CEFC
:107DC0007D907D05C8A5034267010005000052654E
:107DD000747261637473205761726E696E6700EA32
:107DE0007DAE7D0388A603D66600204155584F55C9
:107DF0005420436F6E74726F6C2000067ECE7D003F
:107E0000805280BA0200455849542020202020206A
:107E100020202020202000E27CEA7D0300CD00000D
:107E200020416C742023312020202020202020207D
:107E300000407E7C7F0540CF030000000060000012
:107E400020416C74202023312053776974636820AB
:107E5000005A7E207E0680CE030020416C742023D1
:107E600032202020202020202020007A7E407E0505
:107E700040D1030000000060000020416C7420200D
:107E80002332205377697463682000947E5A7E06FB
:107E900080D0030020416C74202333202020202038
:107EA0002020202000B47E7A7E0540D3030000000D
:107EB0000060000020416C74202023332053776938
:107EC0007463682000CE7E947E0680D20300204139
:107ED0006C7420233420202020202020202000EE3D
:107EE0007EB47E0540D50300000000600000204104
:107EF0006C74202023342053776974636820000851
:107F00007FCE7E0680D4030020416C742023352070
:107F1000202020202020202000287FEE7E0540D732
:107F2000030000000060000020416C742020233515
:107F3000205377697463682000427F087F0680D6EB
:107F4000030020416C742023362020202020202094
:107F5000202000627F287F0540D9030000000060D8
:107F6000000020416C74202023362053776974630D
:107F70006820007C7F427F0680D803004558495422
:107F800020202020202020202020202000207E6271
:107F90007F0300CD00004154206D6F6465202020D8
:107FA00020202020202000B27F048000001E80B608
:107FB000020041542073746570202020202020206E
:107FC000202000CC7F967F05009E02004154207443
:107FD00069636B73202020202020202000E67FB2E0
:107FE0007F05009F0200746F20545A20202020201B
:107FF000202020202020000480CC7F0304DB000010
:10800000000C5C00455849542020202020202020CE
:108010002020202000967FE67F0300CD0000415401
:10802000206D6F6465202020202020496E63003879
:108030008038800000B602004154206D6F646520D6
:108040004F6E652053686F74001E801E800100B65D
:108050000200202020202020204348312020202002
:108060002020006A80128101000020202020202092
:10807000204348322020202020200082805280038C
:1080800000002020202020202043483320202020D2
:108090002020009A806A80050000202020202020D7
:1080A0002043483420202020202000B280828007F6
:1080B00000002020202020202043483520202020A0
:1080C000202000CA809A8009000020202020202043
:1080D0002043483620202020202000E280B2800B60
:1080E000000020202020202020434837202020206E
:1080F000202000FA80CA800D0000202020202020AF
:1081000020434838202020202020001281E2800FC8
:1081100000002020202020202050504D2020202012
:108120002020005280FA80800000202020427564C8
:1081300064792020426F782020200044815E8109EC
:108140008078810020202020205461626C6573209B
:1081500020202020005E812A81098012820045585B
:108160004954202020202020202020202020002AC8
:108170008144810300CD00004D6173746572203F1E
:108180002020202020202020009281C8810300A1EF
:10819000020020204D617374657220204D6F64656C
:1081A000202000AE8178810000E281B70200537484
:1081B0007564656E74203F2020202020202000C898
:1081C0008192810300A002004558495420202020BC
:1081D0002020202020202020007881AE810300CDA7
:1081E00000004D204D6F64653D4D6963726F53749F
:1081F000617200FA81FA810000004D204D6F6465C4
:108200003D46757461626120202000E281E28101B7
:1082100000004169726372616674205461626C652A
:108220002031003282528309866C83DA03DA5CE003
:108230005C004169726372616674205461626C65AE
:108240002032005282128209866C83E503DA5CE0F8
:108250005C00476C6F62616C20205461626C652029
:108260002031007282328209866C834602DA5CE039
:108270005C00476C6F62616C20205461626C652009
:108280002032009282528209866C835102DA5CE0CD
:108290005C00476C6F62616C20205461626C6520E9
:1082A000203300B282728209866C835C02DA5CE061
:1082B0005C00476C6F62616C20205461626C6520C9
:1082C000203400D282928209866C836702DA5CE0F5
:1082D0005C00476C6F62616C20205461626C6520A9
:1082E000203500F282B28209866C837202DA5CE089
:1082F0005C00476C6F62616C20205461626C652089
:108300002036001283D28209866C837D02DA5CE01B
:108310005C00476C6F62616C20205461626C652068
:108320002037003283F28209866C838802DA5CE0AF
:108330005C00476C6F62616C20205461626C652048
:108340002038005283128309866C839302DA5CE042
:108350005C00455849542020202020202020202047
:10836000202000128232830300CD0000504F5320A2
:108370003020202020202020202020200086838ADA
:10838000840100D00000504F5320312020202020B5
:1083900020202020202000A0836C830100D1000039
:1083A000504F532032202020202020202020202029
:1083B00000BA8386830100D20000504F532033203F
:1083C0002020202020202020202000D483A08301F2
:1083D00000D30000504F53203420202020202020A4
:1083E0002020202000EE83BA830100D40000504FEB
:1083F000532035202020202020202020202000086D
:1084000084D4830100D50000504F53203620202013
:108410002020202020202020002284EE830100D66E
:108420000000504F532037202020202020202020E3
:108430002020003C8408840100D70000504F5320C6
:108440003820202020202020202020200056842298
:10845000840100D80000504F5320392020202020D4
:108460002020202020200070843C840100D90000BE
:10847000504F532031302020202020202020202049
:10848000008A8456840100DA0000455849542020AF
:1084900020202020202020202020006C83708403B6
:1084A00000CD000020545820566F6C7420204D657C
:1084B0007465722000C084428607882E5D6667005E
:1084C000545820416C61726D20566F6C7461676501
:1084D00000E084A48408C8B90266670000FF0000B9
:1084E000526573657420426174742054696D6572BD
:1084F00000FE84C084038CDB00E866665D002052C9
:108500005820566F6C7420204D6574657220001AD7
:1085100085E08407884A5D666700536572766F2040
:10852000204D696E2050756C7365003A85FE84029B
:10853000C8AE027867E803881300536572766F202F
:10854000204D61782050756C7365005A851A85023C
:10855000C8B0027867E8038813004E756D626572D3
:1085600020204368616E6E656C73007E853A8505D8
:10857000CEA2028A6704000900125D1A5D00202065
:108580002053796E63207769647468202020009EF0
:10859000855A8502C8A3027867C800DC0500202040
:1085A000536869667420496E76657274202000BA3B
:1085B000857E850388CD039C67002020466F726D01
:1085C000617420466C617368202000D4859E850705
:1085D00080745D0020202020436F6E66696775728D
:1085E0006520202000EE85BA850980BC8600202009
:1085F0004A6F79537469636B2043616C20200008D3
:1086000086D48509807889002020202020202046DB
:108610004D53202020202020002686EE85038CE963
:1086200000D666225D00204672657175656E6379BD
:108630002042616E6420004286088600805C86D1FC
:1086400002004558495420202020202020202020AE
:10865000202000A48426860300CD000020202020B6
:10866000204E6F202052462020202020007486A417
:10867000860000002020202020353020204D487A20
:1086800020202020008C865C8601000020202020F5
:1086900020353320204D487A2020202000A48674E5
:1086A000860200002020202020373220204D487AEA
:1086B00020202020005C868C860300004F7574709B
:1086C0007574206368616E6E656C203100D8860C0D
:1086D00088000126880004004F757470757420634B
:1086E00068616E6E656C203200F486BC86000126DF
:1086F000880104004F7574707574206368616E6E34
:10870000656C2033001087D886000126880204009B
:108710004F7574707574206368616E6E656C20347B
:10872000002C87F486000126880304004F757470BE
:108730007574206368616E6E656C20350048871023
:1087400087000126880404004F75747075742063D7
:1087500068616E6E656C20360064872C8700012688
:10876000880504004F7574707574206368616E6EBF
:10877000656C203700808748870001268806040042
:108780004F7574707574206368616E6E656C203807
:10879000009C8764870001268807040053656C6588
:1087A00063742041696C20205472696D00B8878021
:1087B000870001F688B2020053656C65637420453A
:1087C0006C6520205472696D00D4879C870001F687
:1087D00088B3020053656C65637420527564202071
:1087E0005472696D00F087B8870001F688B4020002
:1087F00053656C6563742054687420205472696DED
:10880000000C88D4870001F688B502004558495409
:1088100020202020202020202020202000BC86F0A6
:10882000870300CD00002020202041696C65726F15
:108830006E2020202020004088DC880100DC000021
:1088400020202020456C657661746F7220202020E6
:10885000005A8826880200DC0000202020202052B8
:10886000756464657220202020200074884088038D
:1088700000DC0000202020205468726F74746C6546
:1088800020202020008E885A880400DC0000202050
:10889000202020202043483520202020202000A810
:1088A0008874880500DC0000202020202020204340
:1088B000483620202020202000C2888E880600DC38
:1088C0000000202020202020204348372020202086
:1088D000202000DC88A8880700DC00002020202061
:1088E000202020434838202020202020002688C235
:1088F000880800DC0000202020204E6F20205472C9
:10890000696D202020200010895E890000DC0000B5
:1089100020202020205472696D203120202020202A
:10892000002A89F6880100DC000020202020205445
:1089300072696D2032202020202000448910890295
:1089400000DC000020202020205472696D2033209C
:1089500020202020005E892A890300DC00002020DE
:108960002020205472696D2034202020202000F621
:108970008844890400DC00002020202041696C65C7
:10898000726F6E2020202020009489908A07803406
:108990005F15040020202020456C657661746F729D
:1089A0002020202000B08978890780345F1B0500D3
:1089B0002020202052756464657220202020202011
:1089C00000CC8994890780345F2106002020202074
:1089D0005468726F74746C652020202000E889B0A0
:1089E000890780665E27070020202020202043483A
:1089F000362020202020202000048ACC8907806691
:108A00005E3B0000202020202020434837202020EB
:108A10002020202000208AE8890780665E3F010030
:108A2000202041696C65726F6E207472696D202020
:108A3000003C8A048A07807A5D2B080020456C651B
:108A40007661746F7220207472696D2000588A20DC
:108A50008A07807A5D2F0900202052756464657250
:108A600020207472696D202000748A3C8A07807A05
:108A70005D330A00205468726F74746C6520207432
:108A800072696D2000908A588A07807A5D370B00E2
:108A900045786974202020202020202020202020BC
:108AA000007889748A0300CD0000202020204365CF
:108AB0006E7465722020202020200000202020528B
:108AC000696768742F446F776E2020200000202093
:108AD00020204C6566742F55702020202020000037
:108AE00001000F00D20000000300D20000001E00B1
:108AF000D2000080120902C802AC0194018A02D09F
:108B000001C4017A02F501C10105002502E1012835
:108B100002DE015E02B5012402E401360173005F4A
:108B2000016F0000000800010409101924314051B0
:108B30006400132433404B545B6063640001020300
:108B4000060C1522334964001B31424F585E6162A6
:108B50006364000A141E28323C46505A64001428EC
:108B60003C5064503C28140000050A0F14192837A3
:108B7000465564000F1E2D3C4B50555A5F64010A48
:108B80000000109001FF00A5E7C009F30000DC051C
:108B90009411010203040000005801000102830443
:108BA00005060708090A0B0C0D0E0F000000000057
:108BB00000000000000000000000000000000000B5
:108BC00000000000000000000000000000000000A5
:108BD0000000000000000000000000000000000095
:108BE0004D4F44454C203031202020202020202093
:108BF000000001B80B00013C190000000001B80B97
:108C000000013C190000000001B80B00013C1900F4
:108C1000000000FEA00F1901D00700FEA00F00FE0B
:108C2000A00F00FEA00F0001B80B000132FF3200C0
:108C300032003200CEFFCE00CE00CE000000001485
:108C4000140000000A0A0000000A0A0000000A0AD4
:108C50000000F4010A0000000A0A0000000A0A00ED
:108C600000000A0A0000000A0A0000000A0A0000C8
:108C7000000A0A0000000A0A000000000000000AC2
:108C800000000000000200000000000000FF0001E2
:108C9000028304050607898B4B8C0D8E8F0100081B
:108CA0001000074B8C0400200000000000FF0D00A6
:108CB00020002000200020002000000104091019DD
:108CC000243140516400132433404B545B6063648F
:108CD0000000000000000000000000000000000094
:108CE0000201030405060708000000000000000060
:108CF0000000000000000000000000000000000074
:108D00000000000000000000000000000000000063
:108D10000000000000000000000000000000000053
:108D20000000000000000000000000000000000043
:108D30000000000000000000000000000000000033
:108D40000000000000000000000000000000000023
:108D50000000000000000000000000000000000013
:108D60000000000000000000000000000000000003
:108D700000000000000000000000000000000000F3
:108D800000000000000000000000000000000000E3
:108D900000000000000000000000000000000000D3
:108DA00000000000000000000000000000000000C3
:108DB00000000000000000000000000000000000B3
:108DC00000000000000000000000000000000000A3
:108DD0000000000000000000000000000000000093
:00000001FF
